:020000040800F2
:1000000000180020E7690008956900085D6A00088B
:10001000996900089B6900089D69000800000000BC
:100020000000000000000000000000009F690008C0
:10003000A169000800000000A36900084910000839
:10004000A7690008A9690008AB690008AD69000844
:10005000AF690008B1690008B3690008B569000814
:10006000B7690008B9690008BB690008BD690008E4
:10007000BF690008C1690008C3690008C5690008B4
:10008000C7690008C9690008CB690008CD69000884
:10009000CF690008D1690008D3690008D569000854
:1000A000D7690008D9690008DB690008DD69000824
:1000B000BD100008E1690008E3690008F55D00086B
:1000C000034B802252049A61024B04221A6070474B
:0800D000000400487C1500202B
:1000D80033230349034A0A60013B002BFBD17047D5
:0800E80000300040AAAA00004C
:1000F000294AD16980239B020B43D3619023DB05FE
:100100001A6850218A431A601A6850310A431A60EB
:100110001A6A22490A401A62196A882252010A435D
:100120001A621F4B1F4A13601F4A13601F4B1B6844
:10013000262B28D00CD9392B2BD0603B5A1E93414B
:100140005B421B4A13409C225201944663440BE0DD
:10015000132B1BD01F3B5A1E93415B42154A134081
:10016000C022D200944663449BB2134A93818023F9
:100170009B025360002393602D3313600F4B80224A
:1001800052051A6070479C23DB00EDE79C231B019E
:10019000EAE7D0239B00E7E700100240FF00FFFFE3
:1001A000FC10002058150020541500208815002050
:1001B00020EEFFFFA0FBFFFF0044004000E100E055
:1001C00004498022CB691A42FCD080B2014B1885C9
:0801D0007047C04600440040E6
:1001D80010B504000D4B1B68002B0AD0023B02220D
:1001E800934310D00A4B1B68002B0ED005F052FE2B
:1001F8000BE0FFF7E1FF064B1B68002B05D0200042
:1002080005F048FE01E0FFF7D7FF10BD6415002098
:040218008814002026
:10021C0010B504003C4B1868C3433C4A1168CA43F0
:10022C000140013165D03A4901200860190C394868
:10023C0001601B041B0C38480360002902D13549AE
:10024C0036480860002B02D1334B35491960D10771
:10025C00C91706230B400A3332490B6032490B6035
:10026C0013065B0E31490B6031490B60002C3FD0FB
:10027C0053059B0F2F490B60D10A1F2001400431FD
:10028C002D4B1960120C2D4B1A602D4B1B68DB4348
:10029C001A04120C2B490A601B0C03402A4A1360E7
:1002AC002A4B2B4C2B48191904CBD2430A6083429E
:1002BC00F9D1294C2948191904CBD2430A6083423D
:1002CC00F9D103F023FE1F4B1B68002B07D09023A2
:1002DC00DB051B8A1B0702D41A4B00221A600D2067
:1002EC00FFF774FF04F0A8F9164B1B68002B05D11F
:1002FC0010BD03F0E7FF002CE3D1F9E7013B184AEE
:10030C00136003F011FBF3E7007400080474000899
:10031C006C150020141500207015002083040000BB
:10032C0040570000D8140020AC1400208815002081
:10033C005C150020B4140020BC140020B81400205C
:10034C000874000810150020841500201074000893
:10035C00F893FF17007A00080888FF170080000840
:04036C00CC1400208D
:1003700010B5114B1B68022219009143012909D0C5
:10038000022B0AD0042B0FD00C4A802311680B4398
:10039000136001E0FFF714FF10BD094B1B68002B31
:1003A000F2D005F07BFDF7E7054B1B68002BEBD087
:1003B00005F0A6FDF0E7C04664150020F01400200B
:0403C000881400207D
:1003C40010B504003034E4B2392C01D93730C4B24A
:1003D4000F4B1B68002B07D002229343012B0ED036
:1003E4002000FFF7EBFE10BD2000FFF7E7FE094BEE
:1003F4001B68002BF7D0200005F04EFDF3E7054BFA
:100404001B68002BECD0200005F046FDEBE7C0464E
:0804140064150020881400208B
:10041C00F0B5C64600B58CB007A9344B0A0013CB17
:10042C0013C203CB03C201A9314B0A0013CB13C275
:10043C0003CB03C2198811809B7893702D4B01223A
:10044C001A602D4B1B68043B5A4253412B4A1360D4
:10045C0004F0D4FE2A4A2B4B1A602B4B98462B4F98
:10046C00284E2B4D06E02B68002B13D1254B1B6817
:10047C00002B0FD043461F6034689442F3D0A30581
:10048C009B0D244922008B42EDD12E20FFF79EFEBE
:10049C002200E8E7184B1B68042B13D007A806F0C2
:1004AC0000FB1B4B1B68002B10D06F20FFF78EFE40
:1004BC006B20FFF78BFEC82000F09CF80CB080BCC2
:1004CC00B846F0BD01A806F0ECFAEAE76520FFF7A4
:1004DC007DFE7220FFF77AFE7220FFF777FE6F2009
:1004EC00FFF774FE7220FFF771FEE4E7D86E000888
:1004FC00EC6E0008181500206415002084140020F0
:10050C00B80B00006015002000300040AAAA0000C3
:08051C0088140020FF03000019
:1005240010B52C4B1B68002B15D12A4B32221A60B4
:10053400294B2A4A1A602A4B1B68002B0CD0013B1A
:10054400274A1360002B07D0264B1B685A1C132B19
:1005540007D0244B1A6010BD234B802252009A61AD
:10056400F2E7204B00221A60204B1B68002B09D1B4
:100574001F4B1B68002BEED1FFF74EFF0D20FFF73A
:1005840029FEE8E71B4B1B68042B0FD01A4B1B6892
:10059400012BE0D104F01CFD174B00221A60FA2055
:1005A400400000F02BF8FFF737FFD4E7124B1B682D
:1005B400002BD0D104F00CFD0F4B01221A60FA205D
:1005C400400000F01BF8FFF727FF0A4B1B68042BC1
:1005D400C1D0DBE76815002000300040AAAA000063
:1005E4007C150020641400200004004888140020B6
:0C05F4001815002064150020841400205D
:1006000010B5054B1860002805D01C00FFF78AFFC5
:0C0610002368002BFAD110BD80150020DB
:10061C00F8B5D1490122CB681A42FCD1CE4B1B69EB
:10062C001B0604D5CC4BCD4A5A60CD4A5A60CA4BF6
:10063C001A6902210A431A61CA4A5A611A693E317F
:10064C000A431A6119000122CB681A42FCD1C24B31
:10065C00DB689B0604D5C04AD36820210B43D360CA
:10066C00BD4B1A6902218A431A611A6901390A437E
:10067C001A61BD4B1B68DB43BA4A1380B649012291
:10068C00CB681A42FCD1B44BDB689B0604D5B24A4A
:10069C00D36820210B43D360B44B1B68DB43B44AB3
:1006AC001380AD490122CB681A42FCD1AA4BDB68FE
:1006BC009B0604D5A84AD36820210B43D360AD4BCD
:1006CC001B685B00FF221A40AB4B1B680A3B591E90
:1006DC008B411A43A94B1B685B02C021C9000B401C
:1006EC001A43A74B1B68043BDB061B0C1343DB4371
:1006FC00A44A138098490122CB681A42FCD1964B2C
:10070C00DB689B0604D5944AD36820210B43D36045
:10071C009D4B1B68DB439D4A13808F490122CB689C
:10072C001A42FCD18C4BDB689B0604D58A4AD368F1
:10073C0020210B43D360964B1B68DB43954A1380F7
:10074C0085490122CB681A42FCD1834BDB689B069E
:10075C0004D5814AD36820210B43D3608E4B1B6890
:10076C00DB438E4A13807C490122CB681A42FCD1B0
:10077C00794BDB689B0604D5774AD36820210B4361
:10078C00D360874B1B68DB43864A13807249012276
:10079C00CB681A42FCD1704BDB689B0604D56E4AC1
:1007AC00D36820210B43D3607F4B1B68DB437F4A0C
:1007BC00138069490122CB681A42FCD1664BDB6875
:1007CC009B0604D5644AD36820210B43D360784838
:1007DC00784C241A604B01222025774F02E004301C
:1007EC00B8421AD006190168C9433180D9680A4247
:1007FC00FCD1D9680D4202D0D9682943D96001686F
:10080C00C943090C7180D9680A42FCD1D9680D42E0
:10081C00E5D0D9682943D960E1E74F4B1A6901212A
:10082C008A431A61654A664911601A6902210A43B2
:10083C001A61644A5A611A693E310A431A611900F5
:10084C000122CB681A42FCD1434BDB689B0604D5D2
:10085C00414AD36820210B43D3603F4B1A690221D4
:10086C008A431A611A6901390A431A6152480122F2
:10087C002025554F02E00430B8421AD00619016801
:10088C00C9433180D9680A42FCD1D9680D4202D0E3
:10089C00D9682943D9600168C943090C7180D968AA
:1008AC000A42FCD1D9680D42E5D0D9682943D960F8
:1008BC00E1E74648464C241A274B01222025454F98
:1008CC0002E00430B84219D006190168C9433180DE
:1008DC00D9680A42FCD1D9680D4202D0D9682943A3
:1008EC00D9604188C9437180D9680A42FCD1D96862
:1008FC000D42E6D0D9682943D960E2E7164B1A6954
:10090C0001218A431A612D4A2D4911601A6902216D
:10091C000A431A61304A5A611A693E310A431A6114
:10092C0019000122CB681A42FCD10B4BDB689B06E9
:10093C0004D5094AD36820210B43D360064B1A69AE
:10094C0002218A431A611A6901390A431A61012288
:10095C002025224F47E0C046002002402301674576
:10096C00AB89EFCD00740008701500201415002021
:10097C000274000888150020D8140020B41400203C
:10098C00BC14002004740008B8140020067400087D
:10099C001015002008740008841500200A74000843
:1009AC00D41400200C740008D01400200E7400081D
:1009BC000808002010740008F80B002000300040DC
:1009CC00AAAA000000780008F80D002008020020F8
:1009DC00007A000808040020007C000808080020A9
:1009EC000430B84219D006190168C9433180D9685E
:1009FC000A42FCD1D9680D4202D0D9682943D9608A
:100A0C004188C9437180D9680A42FCD1D9680D422A
:100A1C00E6D0D9682943D960E2E7064B1A6901216F
:100A2C008A431A611A697F310A431A610A20FFF757
:080A3C00E1FDF8BD00200240BD
:100A440070B5041E00DA9CE0092C00D893E0632CF6
:100A540000D881E0FA239B009C426ED3534B9C4206
:100A64005AD9534B9C4248D9524B9C4236D9524B8B
:100A74009C4224D9514B9C4212D9514B9C4200D9DF
:100A840084E05049200006F0FCFA05004D4920009E
:100A940006F0E9F90C0028003030C0B2FFF79AFBE9
:100AA4004949200006F0EDFA05004749200006F008
:100AB400DAF90C0028003030C0B2FFF78BFB434951
:100AC400200006F0DEFA05004049200006F0CBF9CC
:100AD4000C0028003030C0B2FFF77CFB3C492000FA
:100AE40006F0CFFA05003A49200006F0BCF90C00E4
:100AF40028003030C0B2FFF76DFB3649200006F005
:100B0400C0FA05003349200006F0ADF90C002800B6
:100B14003030C0B2FFF75EFBFA218900200006F0F6
:100B2400B0FA0500FA218900200006F09CF90C00B7
:100B340028003030C0B2FFF74DFB6421200006F0DE
:100B4400A0FA05006421200006F08DF90C002800AD
:100B54003030C0B2FFF73EFB0A21200006F091FAC4
:100B640005000A21200006F07EF90C002800303030
:100B7400C0B2FFF72FFB20003030C0B2FFF72AFBD2
:100B840070BD2D20FFF726FB64425DE7124920006B
:100B940006F077FA05001049200006F064F90C000D
:100BA40028003030C0B2FFF715FB6AE70F270000BA
:100BB4009F8601003F420F007F969800FFE0F505F5
:100BC400FFC99A3B00E1F5058096980040420F006A
:0C0BD400A08601001027000000CA9A3B18
:100BE00070B58CB006AD124B2A0013CB13C213CBD9
:100BF00013C26C460F4B220043CB43C243CB43C2CC
:100C00000D20FFF7E9FA280005F051FF3420FFF727
:100C1000E3FA2E20FFF7E0FA2420FFF713FF20006D
:100C200005F045FF0D20FFF7D7FA0CB070BDC046A8
:080C30007062000888620008F0
:100C380070B552494A6980239B0213434B614A6944
:100C48008023DB0213434B619020C005002303601F
:100C58004B4A13604B4CC4604B48D060D4684B4D32
:100C68002C40D4601068284010601468802040022E
:100C7800204310608020400090618A69FF38024359
:100C88008A6143490A680F3002430A60414A3221A7
:100C98001160414A1360414A1360414A1360414A56
:100CA80041491160414A42491160424A1360424A2F
:100CB8001360424A13600A2241490A6041490A60A6
:100CC800414A13600B2241490A6041490A60414A7E
:100CD8001360414A1360414A1360414B414A1A600C
:100CE800414B1868FA21890006F0C9F901388023B8
:100CF8005B0498420DD23D4A50603D48036A1B028E
:100D08001B0AC02109060B430362002393600733C3
:100D180013600A20FFF770FC364C374B2360374BC3
:100D2800A3600220FFF768FC022363600220FFF73C
:100D380063FC334B23600020FFF76CFA0220FFF7B7
:100D48005BFCFFF7D1F90220FFF756FCFFF744FFE1
:100D58000220FFF751FC2B4B00221A60FFF75AFBC9
:100D68000120FFF757FA284C03F03AF902F01CF873
:100D78002368002BF8D002F03DFEF5E70010024092
:100D880000040048AAAA0AA4AAAAAAAAFFFFFCFF6C
:100D980000000140681500207C1500208015002007
:100DA8006015002014150020830400007015002031
:100DB8004057000084140020181500206C150020EE
:100DC800D8140020AC1400206415002088150020D9
:100DD8005C1500208415002078150020741500206B
:100DE800C4140020A1B0B9120402002010E000E0F1
:100DF80000ED00E00030004055550000FFFF000006
:0C0E0800CCCC000088140020A0140020B6
:100E140010B5FFF785FB0F4B1B680F4A126893420E
:100E240015D05A1C0B490A601B7880200002184315
:100E34000A4B1B689A4207D0094B802252049A61DC
:100E4400084B04221A6010BD074A0A60F4E7002028
:100E5400F9E7C04654150020581500200002002070
:0C0E6400000400487C150020FC10002059
:100E700010B50E4B1B68002B0AD10D4B1B68002BC5
:100E800003D004F0EDFD002801D1FFF7C3FF10BD32
:100E9000023B0222934306D0054B1B68002BF6D081
:100EA00004F0DEFDF3E7FFF7B5FFF0E7641500207F
:040EB0008814002082
:100EB40010B57F2845D90300F03B0D2B03D8484AD1
:100EC400DA40D30716D4F6281CD0F7281AD8454B95
:100ED4001A680F230340511E8B4201D0002A28D1E7
:100EE400414B1860F0231840404B1860404B0122DE
:100EF4001A6006E000233E4A13603B4A13603B4AF3
:100F0400136010BD3B4B1B68990000043A4A88509B
:100F14005A1C1F2B09D0374B1A600023344A136024
:100F2400314A1360314A1360EBE7324B00221A60F6
:100F3400F3E700232E4A13602B4A13602B4A1360F5
:100F4400DFE72B4B1B68002B19D0012B1ED0022B83
:100F5400D7D1284B1A689400234B1B681B042749DC
:100F6400096809020B431843234BE050531C1F2A02
:100F740031D0204A13601E4B01221A60C1E71A4A7D
:100F840013601A4A13601D4A1360BAE71B4B1860BA
:100F9400164B1B6810229343C02B09D0124B1B68BD
:100FA4000E3A9343F12B03D0114B02221A60A8E7A7
:100FB400104B1A6891000C4B1B681B0418430E4B12
:100FC400C850531C1F2A02D00A4A136099E7094BE0
:100FD40000221A6095E7074B00221A60CBE7C0464F
:100FE400B122000084150020601400206C1400203D
:100FF40068140020781500208C1200208C15002025
:1010040010B5FFF78DFA0C4B1B680C4A126893421B
:101014000FD099000A4A8A588020000610435A1CAF
:101024001F2B02D0044B1A6010BD034B00221A6020
:10103400FAE70020F8E7C046741500207815002070
:041044008C120020EA
:10104800164B1B68002B02D0013B144A1360144B4B
:101058001B68002B02D0013B114A1360114B1B681F
:10106800002B02D0013B0F4A13600F4B1B68002B6B
:1010780002D0013B0C4A13600C4B1B68002B02D0BA
:10108800013B0A4A13600A490A6853035A40530C41
:1010980053405A0153400B607047C0466815002002
:1010A8008015002060150020E4140020B0140020F2
:0410B800C41400203C
:1010BC0010B51B4BDB699B062CD5194B9B8C9BB23B
:1010CC00184A126802218A43012A19D0FF221A40B9
:1010DC00022A0FD0042A10D0134A11680B7013681F
:1010EC0001331360114A1268934213D10E4B104A0C
:1010FC001A600FE00F4A1160EEE700F063FD09E0A3
:10110C00094A11680B70136801331360074A12689F
:10111C00934200D010BD044B054A1A60FAE7C04652
:10112C0000440040641500205815002000020020E7
:08113C00FC100020A4140020A7
:10114400024A202311680B4313607047F0140020F7
:10115400064A1368043B1360054A0C32934204D2D6
:10116400044A042311680B4313607047C014002021
:0811740010140020F01400200B
:10117C00084B1A68111D1960074B4033994202D273
:10118C00136853607047054A042311680B431360BE
:10119C00F8E7C046C014002010140020F014002002
:1011AC00044B19680A1F1068096811601B681860E5
:0811BC007047C046C01400207A
:1011C400034A1368191D11601A1F12685A60704788
:0411D400C014002023
:1011D800074A1368190008390868043B1B680B6044
:1011E8001368191F1B680B60136818607047C046A6
:0411F800C0140020FF
:1011FC00074A13681968181F006818601368181FCD
:10120C00083B1B6803601368083B19607047C046B5
:04121C00C0140020DA
:101220000C4B19680A680C4BCB1A9B109B1A042BA9
:1012300006D4002A0AD092008A1A13680B607047FD
:10124000064A042311680B431360F8E70439014B85
:101250001960F4E7C014002010140020F0140020DE
:1012600030B5144B1A681168134BD31A9B105B1AD4
:10127000042B19D4043A0F4B1A60012913D9012306
:101280005B1A9B009D580222521A9200094C236857
:1012900098589B18043B1860013904320029F6D194
:1012A000044B1B681D6030BD044A042311680B43C6
:1012B0001360F8E7C014002010140020F014002080
:1012C000F0B5144B1A681568134BD31A9B105B1BAF
:1012D000042B19D4043A17680E4B1A60012D12D949
:1012E0006E1E0422524200211C00236898589B184D
:1012F00058600131043AB142F7D101235D1B054B1F
:101300001B68AD00EF50F0BD044A042311680B4385
:101310001360F8E7C014002010140020F01400201F
:10132000054B1A68111F12680868844662440A60F7
:0C1330001A68043A1A607047C0140020CC
:10133C00024B1A681368013313607047C014002005
:10134C00054B1A68111F12680868821A0A601A681D
:0C135C00043A1A607047C046C01400201C
:10136800024B1A681368013B13607047C0140020D1
:10137800044B1A681368002B00DB70475B4213604C
:08138800FBE7C046C014002081
:1013900010B50F4B1B681A68D117501848401F280A
:1013A00009DC191F0A4C2160002A0BDB0B000968BD
:1013B0009140196010BD074A8023DB0011680B4380
:1013C0001360F7E7043B1A68C2401A60F2E7C046B0
:0813D000C0140020F0140020FD
:1013D800054B1A68111F1268086802400A601A68EB
:0C13E800043A1A607047C046C014002090
:1013F400054B1A68111F1268086802430A601A68CC
:0C140400043A1A607047C046C014002073
:10141000054B1A68111F1268086842400A601A6872
:0C142000043A1A607047C046C014002057
:10142C00024B1A681368DB4313607047C01400202A
:10143C00024B1A6813685B4213607047C01400209B
:10144C00054B1A68111F1268086842430A601A6833
:0C145C00043A1A607047C046C01400201B
:1014680010B50B4B1C682168002909D0043C206882
:1014780005F0E7FD2060064A1368043B136010BDC1
:10148800044A80231B0111680B431360F7E7C04629
:08149800C0140020F014002034
:1014A00010B50B4B1C68216800290AD0221F106858
:1014B000083C23685843064B1C6005F0C6FD2060BD
:1014C00010BD044A80231B0111680B431360F7E72A
:0814D000C0140020F0140020FC
:1014D80010B50B4B1C682168002909D0043C206812
:1014E80005F0E1FD2160064A1368043B136010BD56
:1014F800044A80231B0111680B431360F7E7C046B9
:08150800C0140020F0140020C3
:1015100070B50D4B1C682568002D0ED0043C266864
:101520002900300005F0C3FD2160074B1C6829002D
:10153000300005F08AFD206070BD044A80231B0145
:1015400011680B431360F7E7C0140020F01400206B
:10155000034A1368191D1160024A12685A607047E5
:08156000C0140020C414002097
:10156800064A1368191F1B6808681B1A584243412A
:101578000B601368043B13607047C046C01400201A
:10158800064A1368191F1B6808681B1A581E8341EE
:101598000B601368043B13607047C046C0140020FA
:1015A800034B1A6811684B424B4113607047C046A1
:0415B800C01400203B
:1015BC00074B1A68131F012112681868904200DC4F
:1015CC0000211960024A1368043B13607047C0463F
:0415DC00C014002017
:1015E00030B5074B1A68111F10680A68D217C40F6C
:1015F0000D68854262410A601A68043A1A6030BD7B
:04160000C0140020F2
:10160400074B1A68131F012112681868904200DB07
:1016140000211960024A1368043B13607047C046F6
:04162400C0140020CE
:10162800064A1368191F1B68086884469C459B4135
:101638005B420B601368043B13607047C0140020C2
:1016480030B5074B1A68111F08681468C20FE517F0
:1016580084426A410A601A68043A1A6030BDC0467A
:04166800C01400208A
:10166C000B4B1B681A680B498A420AD30A498A42F7
:10167C0007D8043B1B681360054A1368083B1360CA
:10168C0004E0064A202311680B4313607047C046E0
:10169C00C014002008080020F80D0020F0140020D1
:1016AC00084B1A68136808498B4205D307498B42CB
:1016BC0002D81B68136004E0054A202311680B4311
:1016CC0013607047C014002008080020F80D00209B
:0416DC00F0140020E6
:1016E000044B0A221A60044B1B68002B01D1034BE8
:1016F0001A607047AC140020F4140020D8140020A5
:10170000044B10221A60044B1B68002B01D1034BC1
:101710001A607047AC140020F4140020D814002084
:1017200006490A681368043A0A60002B05D0044988
:10173000044A0A60013B002BFBD17047C014002013
:0817400000300040AAAA0000DD
:1017480004490B6864221868424303480260043B5A
:0C1758000B607047C0140020B01400208B
:1017640010B5054B1C68221D1A60044B18686421CF
:1017740005F087FC606010BDC0140020B014002088
:1017840030B5094B1B68013B08495B181B041C0C52
:10179400074802681B0E15684B5513689C46614444
:1017A4004C70043A026030BD00150020080200208D
:0417B400C01400203D
:1017B800044B1A68111D1960034B1B68043B1B6816
:0C17C80053607047C0140020C8140020BB
:1017D400024B1B681A68024B1A607047C814002039
:0417E400EC140020E1
:1017E800064B1B681A68002A04D1054A126811685A
:1017F800044A1160043B014A13607047C01400207A
:08180800C8140020EC140020BC
:10181000154B1B68154A19681160154A934218D96F
:10182000144A1268022A07D0043B0F4A1360124A76
:101830001368013B136070470F4A11680F4A126822
:101840009142F1D10D4A002111600A4A0331116021
:10185000EAE7064B00221A60064B1B68022BEAD10E
:10186000044B03321A60E6E7C8140020EC14002091
:10187000C0130020F4010020E01400200C1500200B
:10188000054B00221A605A609A6018000C30034918
:101890000860DA607047C04610140020C0140020B1
:0C18A000014B03221A607047F401002085
:0C18AC00014B01221A607047F40100207B
:0C18B800014B00221A607047F401002070
:1018C40030B50D4B1C68221D1A600C490B685A1C5C
:1018D4000A60587800069A1C0A609A781204024337
:1018E400D81C0860D87800021D1D0D601B791343B5
:1018F4000343636030BDC046C0140020EC140020D4
:10190400054A1368191D116004490A68501C0860CF
:1019140052785A607047C046C0140020EC1400206E
:10192400074B19680A1D1A60064A1368581C106090
:101934005A781201044B9B189B684B607047C04651
:0C194400C0140020EC1400200808002053
:10195000074B1A68511C1960064803685178090141
:10196000054A521819689160043B03607047C046ED
:0C197000EC140020C01400200808002027
:10197C00074B1A68511C196051780902901C1860A9
:10198C0092781143802292050A431A607047C04630
:04199C00EC14002027
:1019A00010B5094B1868021D1A6008490B685A1CCB
:1019B0000A605A7812029C1C0C609B781A438023A0
:1019C0009B051343436010BDC8140020EC14002095
:1019D000084B094A1A60094B1A68511C1960517862
:1019E0000902901C186092781143802292050A43E4
:1019F0001A60704700300040AAAA0000EC140020D2
:101A000010B5094B1B681A68023A80239B051343E3
:101A10001A78722A03D1013B044A136010BD034AAD
:101A20001360FFF7D5FFF9E7C8140020EC1400207D
:101A300010B50A4B1B681B68002B0CD0084A1368B2
:101A4000043B1360074A136803331360034A1368A7
:101A5000043B136010BDFFF7BBFFF7E7C014002085
:081A6000C8140020EC14002062
:101A680010B50A4B1B681B68002B0CD1084A136879
:101A7800043B1360074A136803331360034A13686F
:101A8800043B136010BDFFF79FFFF7E7C014002069
:081A9800C8140020EC1400202A
:101AA00010B5104B1A681100103119600E490B68FF
:101AB000180008380068D060181F00689060186827
:101AC00050600C3B0B6009480368591C0160597851
:101AD00009029C1C04609B78194380239B050B43DF
:101AE000136110BDC8140020C0140020EC140020A5
:101AF00010B5254B1B681A1F1268190008390868B1
:101B00000C3B19685318214A214C146000291DDB35
:101B1000984212DD1C4A1268043A13601D4B1A6881
:101B2000511C196051780902901C18609278114379
:101B3000802292050A431A6010BD134A1368103BB5
:101B40001360144A136803331360F5E7984212DAFE
:101B50000D4A1268043A13600E4B1A68511C196042
:101B600051780902901C18609278114380229205E6
:101B70000A431A60E0E7044A1368103B1360054A01
:101B8000136803331360D7E7C81400200030004007
:081B9000AAAA0000EC140020D9
:101B9800024A1368043B13607047C046C81400200B
:101BA800024A1368103B13607047C046C8140020EF
:101BB80010B5044C23681878FEF70AFB2368043B29
:081BC800236010BDC0140020D1
:101BD00000B583B06A46094B03CB03C2084B1B68B0
:101BE000002B01D003B000BD684604F060FF044B39
:101BF00001221A60034B00221A60F3E7A06200087A
:081C0000F4010020A4140020EF
:101C080000B58FB036220F49684605F056F90E4BDD
:101C18001B681B68102B0DD80C4A1360002B05D0CD
:101C2800094A1368043B13600FB000BD684604F00E
:101C38003AFFF5E7064A8023DB0011680B4313607F
:101C4800F2E7C046786A0008C01400208415002016
:041C5800F014002064
:101C5C0010B5114B1B68002B12D0104B1B78002BAE
:101C6C000ED00F4B1B68002B15D00E4A1368191D94
:101C7C0011600D4A12785A60094B00221A600AE072
:101C8C00FFF7F0F80028FBD0064B1A68111D1960FD
:101C9C00FF231840506010BDF40100209F15002058
:0C1CAC00A8140020C01400209E15002089
:101CB80010B50E4B1B68102B08D00D4B1B6818680D
:101CC800E0231B06C2180B4B9A420CD8084B1B6822
:101CD800186805F0AAF92020FEF77AFA044A136872
:101CE800043B136010BDFEF7A9FEF4E7AC14002016
:081CF800C0140020FF0B0630B0
:101D000010B5064C2368186805F093F92020FEF7FB
:101D100063FA2368043B236010BDC046C014002052
:101D2000F0B587B003AA2A4B13CB13C2294B1A680C
:101D300001929A8801AB9A805B20FEF74DFA264B00
:101D40001B68264A0C3293420DD0244A0C3293422F
:101D50000DD3224A0C32934216D9204C103404255C
:101D60001E4F160024E001A804F0A1FE0CE003A819
:101D700004F09DFE194B00221A605A609A60180008
:101D80000C3015490860DA605D20FEF725FA202046
:101D9000FEF722FA07B0F0BD206805F04AF92020CE
:101DA000FEF71AFA01350C4B1B680434B342EBD929
:101DB000DB1B9B10AB42E7D32020FEF70DFA084B4C
:101DC0001B68102BE8D02068FEF73CFEE7E7C04612
:101DD000C86A0008D46A0008C0140020101400204B
:041DE000AC1400201F
:101DE400F0B5D6464F464646C0B584B001AA394B35
:101DF40003CB03C21B7813702020FEF7EBF9364B9C
:101E04001B68002B5BD0354D00270026C0231B0523
:101E14009946334B9A46304B984616E02020FEF7FD
:101E2400D9F914E06B684A46134221D12020FEF709
:101E3400D1F92020FEF7CEF901360137052F34D829
:101E4400103543461B68B34237D9092EE6D9300012
:101E5400FEF7F6FD3A20FEF7BDF92C00083C207889
:101E64000028DFD0FEF7B6F90134AC42F7D1D9E748
:101E740001A804F01AFE53461B68102B11D02868E1
:101E8400FEF7DEFD2020FEF7A5F94020FEF7A2F9BB
:101E94002804000C05F0CBF82920FEF79BF9023743
:101EA400C4E7286805F0C3F8ECE70D20FEF792F9C3
:101EB4002020FEF78FF90027C2E7002F05D104B0D8
:101EC400E0BCBA46B146A846F0BD0D20FEF782F943
:101ED400F5E7C046C06D0008DC140020100800209F
:041EE400AC1400201A
:101EE80010B5044C2368186804F00FFE2368043BFF
:081EF800236010BDC01400209E
:101F000010B5044C23681878FEF732FA2368043BB6
:081F1000236010BDC014002085
:101F1800F8B50D4A13681F68043B1360002F0CD0F6
:101F28000124E41BA4003D0016003368185DFEF789
:101F38001BFA013D0434002DF7D1034BBF001A688A
:0C1F4800D71B1F60F8BDC046C01400206D
:101F5400F0B5C64600B582B06846214B020012CBEC
:101F640012C204F0A2FD0D20FEF734F91D4DF82332
:101F74009B009846A8440026012723E0FEF72AF98F
:101F84000134285D0028F9D1062C05D82020FEF75D
:101F940021F90134072CF9D12320FEF71BF938006D
:101FA40004F099FD2020FEF715F92020FEF712F920
:101FB4002020FEF70FF901370136052E07D008352A
:101FC400A84509D02020FEF705F90024D9E70D2003
:101FD400FEF700F90026F2E702B080BCB846F0BD77
:081FE400A862000898650008DE
:101FEC0070B5FEF73FFF041E00D1D8E0C0B2704BB5
:101FFC001B68002B08D06F4B1B78002B04D06E4B4A
:10200C0018706E4B01221A600A2800D1C4E0022815
:10201C0000D8C3E0674B1B78002B08D109281FD0D0
:10202C00674A12683F2A02D9202800D19EE028284E
:10203C0018D02F2840D01B2868D10024002B00D1A9
:10204C00ADE00E38FEF7C2F85D4B1A685D4B2021EF
:10205C0099549B18002159705B4B1A6002349EE016
:10206C001730DDE7594B1C68002C01D0002496E09A
:10207C00FEF7ACF8FEF7F6FE0028FBD0C0B2202825
:10208C000BD04F490B684F4A2825D554D2185070A5
:10209C0002330B60FEF79AF881E0494B1B68013361
:1020AC004A4A13601838FEF791F82020FEF78EF894
:1020BC000820FEF78BF872E0444B1C68002C01D012
:1020CC0000246CE0FEF782F8FEF7CCFE0028FBD073
:1020DC00C0B22F280BD03A490B683A4A2F25D55459
:1020EC00D218507002330B60FEF770F857E0344B87
:1020FC001B680133354A13602738FEF767F8202038
:10210C00FEF764F80820FEF761F848E0092848D08B
:10211C00122848D0082817D12C4B1D680024002DFC
:10212C003DD1274B1C68002C39D0013C1C60254B41
:10213C0020221A55FEF74AF82020FEF747F808200F
:10214C00FEF744F82C002AE00D2817D11C4B1B6815
:10215C00002B0BD11A4B1A681A4B202199549B183F
:10216C0000215970184B1A60012418E0174B1B689A
:10217C00012BEFD00D20FEF729F8EBE7134B1C6871
:10218C00002C12D10E4D0F4B2A689854FEF71EF8F6
:10219C002B6801332B6002E0002400E000242000B7
:1021AC0070BD0324FBE70424F9E70024F7E7C046DD
:1021BC00F40100209F1500209E150020A81400207B
:1021CC009C1400200C130020A0140020F8140020F4
:1021DC0010B5154B1968154B5A5C202A09D14B1CAC
:1021EC001248013819000133C25C202AFAD00E4B78
:1021FC0019600023002A10D00C4840180C4CC25C0B
:10220C00202A03D01A5501330F2BF8D1084A00208D
:10221C00D0545B18074A136010BD054B00221A708E
:10222C00044B1960F8E7C046941400200C130020EE
:08223C00701300209C14002027
:10224400F0B5DE46474680B587B00E0002AA0024EA
:1022540005E0002B1BD001340132102C08D0035DA3
:102264001370190061391929F3D8203B1370F2E770
:10227400002302AAD37313782D2B0ED1254B0022F1
:102284001A6001239B460127012C0FD82CE0002360
:1022940002AAD37313782D2B2CD01E4B00221A6064
:1022A40000239B4600270120002C2DD0194B1D68CC
:1022B400B84602AB9C46E044002301934346187899
:1022C400310004F046FC431C18D075432D18013727
:1022D40001239C46E0440193A742EFD30D4B1D60BC
:1022E40001205B46002B0FD00A4A13685B4213603F
:1022F400012009E00020012CC0D105E0019B002B46
:1023040001D0044B1D60002007B0C0BCBB46B046E2
:08231400F0BDC0469814002042
:10231C0010B5344B187800285AD0002331490133BA
:10232C005A5C002AFBD12D280FD0302829D12D4AF8
:10233C00527820218A43582A11D02B4A116810292F
:10234C003AD1082B48D900204BE0012B3AD0264A31
:10235C00116810292AD00B2B3ED9002041E0214ACC
:10236C0092782D2A09D00A2B2ED81E481021023023
:10237C00FFF762FF431E984133E00B2BF5D9002089
:10238C002FE02528D9D1174A52782D2A09D00B2BAA
:10239C001CD814480A210130FFF74EFF431E984108
:1023AC001FE00C2BF5D900201BE000232D28C8D1F1
:1023BC00092B11D9002014E02D28CCD000200A2B99
:1023CC000FD809E000200CE000200AE0002008E013
:1023DC00054B19681029E8D00248FFF72DFF431E62
:0C23EC00984110BD70130020AC140020BC
:1023F800F0B51A4C00251A4E0021635C8A5D18005E
:10240800613819280DD8203BDBB210006138192833
:1024180011D8203AD2B2934219D101310829ECD10E
:1024280015E01000613819280DD918002038471E0A
:10243800B84140420340934209D1002AEDD1094BEB
:102448001D600120F0BD203AD2B2202BE3D1013526
:1024580008347D2DD0D10020F4E7C04690650008EF
:0824680070130020CC140020C9
:1024700070B51A4B1B78002B29D0194A00231E0077
:10248000013310321100103909780029F7D1731C7B
:102490001FD03301114C1C19124D16E08B4211D183
:1024A00000290BD00132082A0CD0A15C535D180022
:1024B00061381928F2D8203BDBB2EFE70A4B1E60E7
:1024C000012070BD103C013E05D30022EDE7002045
:1024D000F7E70020F5E70020F3E7C04608080020F2
:0C24E0001808002070130020CC1400200D
:1024EC0010B50F4B1A680F4B1A60FFF771FEFFF710
:1024FC00B9FF002805D00C4B1B6801330B4A136045
:10250C0010BD0B4B1B78302B05D00A4A21231168C8
:10251C000B431360F4E7054B00221A60F0E7C0464A
:10252C009C14002094140020CC14002010150020C2
:08253C0070130020F0140020D0
:10254400074A13680749C85401331360064A934283
:1025540004D9064A202311680B4313607047C04610
:102564000015002008020020FE050000F0140020E1
:1025740010B5144B18688200134BD3581A030AD4AD
:10258400124A1268002A13D19B030BD48000104B0B
:10259400C358984705E00F4A80239B0011680B43FA
:1025A400136010BD0B4A082311680B431360F8E74E
:1025B400DB0304D58000064BC3589847F1E7FFF7C7
:1025C400BFFFEEE7CC1400209C630008F414002045
:0825D40000000020F0140020BB
:1025DC0070B594B00CA9414B0A0013CB13C213CBAA
:1025EC0013C203CB03C205A93D4B0A0013CB13C284
:1025FC0013CB13C21B7813706A463A4B13CB13C21E
:10260C0011001A680A601B790B71374B1B68522B2F
:10261C0009D95224354E344DA05DFDF7D7FD013458
:10262C002B68A342F8D85223314A1360314A002157
:10263C001160314A13602E4D304E03E02C4B1A685A
:10264C002D4B1A60284C2B682268934234D2FFF72A
:10265C00BFFD3378002BF6D0FFF75AFE00280BD0C5
:10266C00274B1A68274B1A60274B1B78002BE5D099
:10267C00264B01221A60E1E7FFF7B8FE002811D0C3
:10268C00234B1B689B00234A9B585B0321D5FFF708
:10269C006BFF214B1B68002B08D1154B1A68164B8E
:1026AC001A60CFE70CA804F0FCF905E01A4B0022E5
:1026BC001A60684604F0F5F90D20FDF787FD5223EA
:1026CC00094A13600A4A13600A4B00221A6014B0BC
:1026DC0070BD05A804F0E5F9EEE7C046D86D00081A
:1026EC00F86D0008146E0008A01400200C130020D4
:1026FC009C140020F8140020941400207013002067
:10270C0098140020041500209F15002008150020A7
:0C271C00CC1400209C630008F014002086
:1027280070B56C20FFF70AFF0C4D2C68FF20FFF7EF
:1027380005FFFF20FFF702FF2B68013B084A9B18A3
:102748001B04180C074909681B0E0D6853550B68C4
:102758009C46624450700C6070BDC0460015002055
:0827680008020020C01400204B
:1027700010B56D20FFF7E6FE064A1368191D1160BB
:10278000054A12685A60FF20FFF7DCFEFF20FFF7C2
:0C279000D9FE10BDC01400200015002070
:10279C0010B57120FFF7D0FE064A1368191D1160A1
:1027AC00054A12685A60FF20FFF7C6FEFF20FFF7AC
:0C27BC00C3FE10BDC0140020001500205A
:1027C800F8B57220FFF7BAFE104E33681D68013560
:1027D8000F4C2D19280AFF273840FFF7AFFE3800A5
:1027E8002840FFF7ABFE0B4B1B68013B1B193268F7
:1027F800190A106821541268A41863707420FFF72E
:102808009DFE3368043B3360F8BDC046C014002009
:08281800080200200015002059
:1028200010B51F4B1B68002B17D11E4B1B681E4A8F
:10283000196811601D4A93422ED91D4A1268022A56
:102840001DD0043B174A13601A4A1368013B1360FA
:10285000194B1A68194B1A6010BD6120FFF772FE00
:1028600000220F4B1A6016490B6801330B601B01E5
:1028700014495A54144B1A68144B1A60E8E70D4A6D
:102880001168134A12689142DBD1114A002111608C
:10289000074A03311160D4E7034B00221A60D7E7DF
:1028A000F4140020C8140020EC140020C0130020F1
:1028B000F4010020E0140020D8140020AC14002003
:1028C000DC1400200808002000150020FC14002063
:0428D0000C150020C3
:1028D40070B5324B1B68002B27D1314B1B681C7819
:1028E40023005C3B022B16D97D20FDF773FC2020CE
:1028F400FDF770FCFFF712FA25006D3D072D15D981
:10290400713C012C1CD9032D0FD8264B1B68188849
:1029140004F057FB09E0244B186801300005000D52
:1029240004F04FFB2920FDF755FC70BD2020FDF776
:1029340051FC5220FDF74EFC3A20FDF74BFCDFE73B
:10294400184B1A68194BD31A082BEED90C3A108875
:1029540004F037FB2020FDF73DFC2020FDF73AFC76
:10296400104C2368083B188804F02BFB2020FDF74B
:1029740031FC6920FDF72EFC2368043B188804F021
:1029840020FB2020FDF726FC7820FDF723FC23689C
:102994001888013004F015FBC7E7C046F014002086
:1029A400E8140020C8140020EC140020C0130020F8
:1029B400204B186800281BD11F4B1B68002B0BD021
:1029C4001E4B1B681E4A1268934205D0D01A9342CC
:1029D4000DD3981AC4300AE01A4B1B681A4A1268BD
:1029E400934204D0D01A934201D3981AC43070474A
:1029F4000238022398430CD00F4B18680028F6D0F5
:102A04000E4B18680E4B1B68984211D00DD2181A41
:102A1400EDE70C4B1B680C4A12689342E7D0D01ABE
:102A24009342E4D3981AC430E1E7C01AC430DEE715
:102A34000020DCE764150020881400202415002001
:0C2A440028150020541500205815002013
:102A500010B5094B1C68221D1A60084B1B68002B1F
:102A600006D0074B1B78002B02D0064B186801E0FC
:102A7000FFF7A0FF606010BDC0140020F40100202B
:082A80009F150020A81400209E
:102A880010B50B4B1C6800230A4909190A48CA5C8F
:102A9800222A03D01A5401334E2BF8D1064A222198
:102AA800D15401330021D154E318044A136010BDF6
:102AB800941400200C130020701300209C14002094
:102AC8001A4B1B185A781300613B192B03D8203A6C
:102AD8001300373B05E02F2A1BD91300303B092B85
:102AE800F6D80F2B18D8114A1018827811006139BE
:102AF800192907D8203A373A11000F2912D8180196
:102B0800401870472F2A0AD9110030390929F4D9F9
:102B1800F1E701204042F4E701204042F1E70120BB
:102B28004042EEE701204042EBE7C0467013002028
:102B3800F0B5C64600B50700404B1B680133404A54
:102B48001360FFF79DFF002600243E4A03E001368C
:102B58000134502C10D0A35C5C2BF8D0222BF7D179
:102B6800384B00221A55384B1D68002D0CD1354CB6
:102B7800364B98461E003BE0354A022311680B434A
:102B8800136080BCB846F0BD012F0ED06320FFF75C
:102B9800D5FC304A13687600A41B2F49CC54013366
:102BA80013600024274D2E0009E06220FFF7C6FCC1
:102BB800EFE7FFF7C3FC0134335D002BE1D0285D5C
:102BC8005C28F6D12000FFF77BFF431C03D00334B9
:102BD800FFF7B4FCF0E71E4A022311680B431360A9
:102BE800CFE7FDF7F5FA0135164B5B5D002BC8D032
:102BF800605D5C2807D0012FF3D03368002BF2D03A
:102C0800FDF7DAFAEFE72800FFF75AFF431C0AD06E
:102C18000335012F0DD043461B68002BE4D0C0B20A
:102C2800FDF7CAFAE0E70A4A022311680B4313606A
:102C3800A7E7C0B2FDF7CCFAD6E7C0469C1400203F
:102C48009414002070130020F41400206415002050
:0C2C5800F01400200015002008020020ED
:102C640010B50F4B1B68032B04D00D4B1B68042BB2
:102C740009D010BDFEF7CCF80028F6D0FF23184089
:102C8400FEF716F9F1E7074B1B68002BF1D002F0B1
:102C9400E5FE0028EDD0FF231840FEF709F9E8E728
:082CA4006415002088140020D3
:102CAC0010B5304B1B68012B0BD0022B1ED0032B05
:102CBC0039D0042B33D02C4A402311680B431360BA
:102CCC0010BD2A4B19680A1D1A60294B1B68294A2A
:102CDC001268934203D005D2D31A4B60F0E700235D
:102CEC004B60EDE79B1AC4334B60E9E7224B1B6842
:102CFC00002BE0D01D4B19680A1D1A601F4B1B6876
:102D0C001F4A1268934203D005D2D31A4B60D7E7FF
:102D1C0000234B60D4E79B1AC4334B60D0E7164BAF
:102D2C001B68002BC7D0FFF797FFFFF795FFFFF746
:102D3C0093FF0E4B1A68111D1960124B1968124B38
:102D4C001B68994203D005D25B1A5360B8E7002385
:102D5C005360B5E7094B1968094B1B685B1A2033A4
:102D6C005360ADE764150020F0140020C01400205F
:102D7C00541500205815002088140020241500201C
:0C2D8C0028150020741500207815002088
:102D980010B5044B1B68022B00D810BDFFF75EFF6F
:082DA800FBE7C04664150020A2
:102DB00010B50023064A1360064A1360064A1360E2
:102DC000FFF7EAFFFFF712F90028F9D010BDC0465F
:0C2DD0009C140020A0140020F814002027
:102DDC0010B5FFF7DBFF154B1B68022B17D0144BFC
:102DEC001868002817D0134B1B780020002B12D02A
:102DFC00FFF7DAFD00280ED0FFF7F2F801280BD010
:102E0C0002280CD00C4B1868431E984103E0074B6A
:102E1C0000221A60012010BDFFF7DAFBF2E7064A28
:102E2C0080235B0011680B431360EBE7A4140020B4
:0C2E3C00F40100209F150020F01400207D
:102E480010B5264B1B68012B0BD0022B1AD0032B75
:102E580031D0042B2BD0224A402311680B43136036
:102E680010BDFDF7D3FF002804D1FFF7B3FF0028FA
:102E7800F7D0F5E71B4B1A68111D1960FF2318409E
:102E88005060EDE7184B1B68002BE4D002F0E4FD1E
:102E9800002804D1FFF79EFF0028F7D0E0E7114B88
:102EA8001A68111D1960FF2318405060D8E70E4BAF
:102EB8001B68002BCFD0FEF7A1F8002806D1FFF73A
:102EC800CDFEFFF787FF0028F5D0C9E7054A13684C
:102ED800191D11600002000A5860C1E7641500203E
:0C2EE800F0140020C0140020881400200A
:102EF40010B5094A1368094918680860043B13604F
:102F04000C002368002B05D0FDF70AFBFFF764FFD4
:102F14000028F6D010BDC046C0140020E4140020E0
:102F240010B5044B1A68642311684B431360FFF710
:082F3400DFFF10BDC0140020F6
:102F3C00134A13681868043B136011281DD0F02342
:102F4C000340A02B0AD00E280AD9B12814D00D4A60
:102F5C008023DB0011680B4313600DE0913B18409C
:102F6C00831E012B02D9063B042B05D8054A80236E
:102F7C00DB0011680B4313607047B120FCE7C046BF
:082F8C00C0140020F014002025
:102F940070B5FFF7D1FF144B1B68002B14D10F2819
:102FA40013D844000322A2409023DB05D96891433F
:102FB400D9601968914319601D6801221100A1406C
:102FC4002943196082409A6170BD084BDA680C216C
:102FD4008A43DA601A688A431A601A6808390A430D
:102FE4001A6002229A61EFE7F014002000040048FE
:102FF40070B5FFF7A1FF154B1B68002B15D10F28E7
:1030040014D844000322A2409023DB05D9689143DD
:10301400D9601968914319601D6801221100A1400B
:1030240029431960103082409A6170BD084BDA68F8
:103034000C218A43DA601A688A431A601A680839CC
:103044000A431A60802292029A61EEE7F01400208B
:04305400000400482C
:1030580010B5FFF76FFF124B1B68002B11D10F281B
:1030680010D84000032282409023DB051968914361
:103078001960D9689143D960D968012282400A430E
:10308800DA6010BD074B1A680C218A431A60DA68A7
:103098008A43DA60DA6808390A43DA60F1E7C04639
:0830A800F014002000040048B0
:1030B00010B5FFF743FF124B1B68002B11D10F28EF
:1030C00010D84000032282409023DB051968914309
:1030D0001960D9689143D960D968022282400A43B5
:1030E000DA6010BD074B1A680C218A431A60DA684F
:1030F0008A43DA60DA6804390A43DA60F1E7C046E5
:08310000F01400200004004857
:1031080010B5FFF717FF0D4B1B68002B0CD10F28CC
:103118000BD84000032282409023DB0519689143B5
:103128001960D9689143D96010BD054B1A680C2104
:103138008A431A60DA688A43DA60F5E7F0140020F7
:043148000004004837
:10314C0010B5FFF7F5FE104B1B68002B0FD10F28A5
:10315C000ED89023DB051B8A0122824013400B49B9
:10316C000A68101D0860002B0AD00123536010BDA3
:10317C00074B1B8A0F2210400E3A82401340EEE799
:10318C0000235360F3E7C046F0140020C014002065
:04319C0000040048E3
:1031A00010B5144BDA6814490A40DA609969802234
:1031B00092000A439A61FCF78FFFFCF78DFFFCF742
:1031C0008BFFFCF789FF0D4B802212061A6100224B
:1031D000DA600B490A6004325A619A6801210A4395
:1031E0009A60190001220B681A42FCD0FCF774FFA8
:1031F00010BDC04600100240FFFDFFFF002401404B
:04320000082701405A
:103204000C4B1A6801210A431A609A6801310A4377
:103214009A60190001228B681A42FCD1064B9A6904
:1032240006490A409A61D968802292000A43DA600A
:103234007047C0460024014000100240FFFDFFFF1C
:10324400F0B589B004AA4F4B13CB13C21B8813806B
:103254006A464D4B13CB13C21B7813704B4B1B6840
:103264001C68621C18D0072C03D92300A03B072B31
:103274001BD8474B9B699B051ED5464B464A1A6093
:103284000F232340590003228A40072B00D971E001
:103294009900424841588F46043B3C4A1360FFF76B
:1032A400AFFF684603F001FC35E03D4A8023DB00B4
:1032B40011680B4313602EE0FFF770FF04A803F0BE
:1032C400F4FBDAE79021C905086810430860C86870
:1032D4009043C86001229A4013002E4A9362042648
:1032E400002714000425A3682B43A36023681D4210
:1032F400FCD0236CFF18FCF7EDFE013E002EF2D14A
:10330400224B1B68BA081A60BB0704D51F4B1A6806
:1033140013680133136009B0F0BD9021C905086832
:1033240010430860C8689043C860D3E79021C9057A
:10333400086810430860C8689043C860CAE79021D1
:10334400C905086810430860C8689043C860C1E7AD
:103354009021C905086810430860C8689043C86094
:10336400B8E79021C905086810430860C86890430D
:10337400C860AFE70A4A8023DB0011680B4313607F
:10338400C9E7C046306E0008406E0008C014002033
:103394000010024000240140FF070000B062000852
:0433A400F014002001
:1033A80010B5074A1368191D1160064A12685A6059
:1033B800FF20FFF7C3F8FF20FFF7C0F810BDC04695
:0833C800C014002000150020D4
:1033D000F8B5104E33681D6801350F4C2D19280AB9
:1033E000FF273840FFF7AEF838002840FFF7AAF86B
:1033F0000A4B1B68013B1B193268190A10682154DB
:103400001268A41863707320FFF79CF83368043BBC
:103410003360F8BDC0140020080200200015002011
:1034200070B57C280DD8C0000E4D441908352D18F4
:103430002078002804D0FCF7CFFE0134AC42F7D14D
:1034400070BD7F2528400001074D441908352D180F
:1034500020780028F4D0FCF7BFFE0134AC42F7D14D
:0C346000EEE7C046906500080808002058
:10346C0070B50001064D441908352D182078002838
:10347C0004D0FCF7ABFE0134AC42F7D170BDC046B2
:04348C00080800200C
:10349000F0B5C64600B582B0A34B1A6800929B886F
:1034A0006A469380A14B1D68002D03D002B080BCFA
:1034B000B846F0BD9E4B1B689E4A13601B78984629
:1034C0001F009D4B1B685E00F6180D20FCF784FE64
:1034D000002E06D02C002020FCF77EFE0134A642F0
:1034E000F9D1944B188803F06EFD2020FCF774FE90
:1034F000404603F068FD2020FCF76EFE7D2F1AD8B1
:103500004046FFF78DFF682F53D0692F57D06A2FA1
:1035100000D182E06B2F00D187E06C2F56D06E2F48
:1035200000D18AE06F2F00D18DE0022342469A43FA
:10353000702A4BD059E02D20FCF74EFE3E20FCF7C0
:103540004BFE2020FCF748FE4046FFF769FF784B12
:103550001B685B787F241C40662F00D19EE0672F9C
:1035600000D1A5E0612F00D1B7E0744C032D00D14C
:10357000C7E02368022B00D8C3E0FCF7D3FFFFF7B6
:1035800019FA0028F2D0FEF731FD0500012800D11C
:10359000ADE0022800D1ADE00428E7D1664B1B68FE
:1035A000002B00D1ADE0664A1360644B02221A6022
:1035B000DCE7644B1B681B68002B07D0C7E7614B37
:1035C0001B68191F1A680B689A42C0D0684603F03E
:1035D0006EFA574B1B68587800029B7818430130ED
:1035E00003F0F1FC2920FCF7F7FD652F35D1504B96
:1035F0001B685C782820FCF7EFFD534B1B68102BF1
:1036000027D02000FDF71EFA2920FCF7E5FD484BE6
:103610001B685B787F241C40A1E74A4B1B681A1F7C
:1036200012681B689A42D1D291E7464B1B681A1F59
:1036300012681B689A42C9D989E7424B1B681B680C
:10364000002BC3D083E73F4B1B681B68002BBDD109
:103650007DE7200003F0B7FCD6E7642F00D076E7C3
:10366000334B1A6893781B04517809060B43117980
:103670000B43D47824021C432820FCF7ADFD324BC9
:103680001B68102B06D02000FDF7DCF92920FCF781
:10369000A3FD67E7200003F096FCF7E72820FCF77E
:1036A0009BFD2000FFF7E2FE2920FCF795FD5CE77B
:1036B0002820FCF791FD2000FFF7D8FE4020FCF702
:1036C0008BFD20010830214C00190004000C03F090
:1036D000B0FC2920FCF780FD47E72020FCF77CFDAB
:1036E0003C20FCF779FD2D20FCF776FD3DE7FEF749
:1036F00075FF3BE70D4A80235B0011680B431360A5
:10370000D4E62020FCF768FD43465C3B022B03D83F
:10371000684603F0CCF9C9E67B20FCF75DFD20206C
:10372000FCF75AFDC2E6C0460C6B0008F0140020FE
:10373000EC140020E8140020E0140020F401002024
:103740000C150020C0140020AC1400200808002034
:1037500010B5FFF79DFE074B1B68002B08D1064BE9
:103760001B681B789B00054A9B589847FFF7B2F8E7
:1037700010BDC046F0140020EC1400200000002012
:1037800010B51B4A1368013313601A4B1A68111DD8
:10379000196019490B6853601A787F2313401B0185
:1037A000164AD3189B680B601B787C2B0BD8144AE5
:1037B0001268032A04D09B00124A9B58984710BDF8
:1037C000FFF7C6FFFBE70E4B1B68032B06D00E4B23
:1037D0001B68002BF3D1FFF7D3FFF0E7FFF758FE8C
:1037E000094B1B68002BEAD1FFF774F8EFE7C046DE
:1037F000E0140020C8140020EC1400200808002069
:0C380000F401002000000020F014002063
:10380C00F0B587B001AA3D4B13CB13C211001A6857
:10381C000A601B790B713A4C3A4BE4183A4B1B6813
:10382C00A34265D2394D384E2F003DE0FEF7CAF960
:10383C0041E0FFF79FFF28E0FFF7B6F800280CD116
:10384C0033681B787C2B1BD8304A1268032A14D09F
:10385C009B002F4A9B58984717E0FEF7C1FB0128A5
:10386C0008D00228ECD12B4A80235B0011680B4353
:10387C0013603DE0FEF7ACFEE2E7FFF763FF04E008
:10388C003B68032B21D0FFF775FFFFF77FFA214B25
:10389C001B68002B2CD11C4B1B68002B1AD001333E
:1038AC00194A1360A34223D22B68002BC4D11A4BA4
:1038BC001B68042BBAD0144B1B681B787C2BB8D814
:1038CC009B00134A9B589847DFE7FFF7DBFDFEF799
:1038DC00FBFFD8E70D4B1B68032B0BD00B4B0122C6
:1038EC001A6000230D4A13700D4A13600D4A1360C1
:1038FC0007B0F0BD01A803F0D4F8EFE7586E00084C
:10390C0008020020F80D0020EC140020F401002027
:10391C0000000020F0140020A41400209F150020AB
:08392C0008150020E014002042
:10393400F8B5274B1C68002C2ED1264B1B681901A7
:10394400254A5218D168C022120511420AD0234ACE
:103954001168081D10601B011F4AD3189B684B6037
:103964002000F8BD1B011C4AD3189A681C4B1A602E
:103974001C4B01221A701C4D2F681C4C26685223C4
:103984002B6023601A4B00221A60FFF73DFF2F6063
:103994002660184B1C68E3E70E4B186802010E4BB7
:1039A4009B18DA68C0231B0514001C401A4204D17A
:1039B40080231843FEF7C4FDD2E76620FEF7C0FD5E
:1039C400044B1868FEF7BCFD0A4B1C68C8E7C046E8
:1039D400F4140020CC14002008080020C014002097
:1039E400EC1400209F150020A01400209C1400203B
:0839F400F8140020F01400207B
:1039FC0070B50023384A1370384A1360384A136084
:103A0C001500384E0EE0384B1B68FF2B24D8652070
:103A1C00FEF792FD344B1868FEF78EFD304B1A689A
:103A2C002E4B1A60314C2B682268934230D2FEF731
:103A3C00CFFB3378002BF6D0FEF76AFC00281FD0A2
:103A4C002B4B1B68002BDED12A4A1368191D116001
:103A5C00254A12685A60E1E76420FEF76DFD224C9E
:103A6C0003202056FEF768FD0223E05EFEF764FD9E
:103A7C0023681812FEF760FD2068FEF75DFDCDE7A8
:103A8C00FEF7F0FC002809D0FFF74EFF002800D00D
:103A9C0070BD134B1A68114B1A60C3E7FEF7A6FCF6
:103AAC0000280AD0FEF760FD134B1B68002BEFD1EA
:103ABC000B4B1A68094B1A60B4E70F4A01231168C3
:103ACC000B4313600D4B1A680D4B1A60044B1A68AC
:103ADC00024B1A60DCE7C0469F15002094140020AE
:103AEC009C1400207013002098140020A0140020B7
:103AFC00F4140020C0140020F0140020FC1400204A
:043B0C000015002080
:103B1000F0B5DE4657464E464546E0B591B00BA996
:103B2000B94B0A0013CB13C203CB03C206AAB74B8F
:103B300013CB13C211001A680A609A888A809B7995
:103B40008B7102AAB24B13CB13C21B881380B14BEB
:103B50001A68B14B1A60FEF741FBFEF789FC00289A
:103B60000DD1FEF749FC002805D1AC4A01231168AC
:103B70000B43136018E10BA802F099FF14E1A54B69
:103B80001A68A54B1A6006A802F091FFA44D2B6895
:103B90001801A44C001903F04CFA0D20FCF71CFB93
:103BA0002B681A01A418E168C02212050800104011
:103BB0000190114200D0FEE01B019A4AD3189C6884
:103BC000994BE41A2405240D1B5D0125612B00D1BE
:103BD000D1E0954E24E00D20FCF7FEFA019D1FE098
:103BE000914B1A195078000202341F5D07432820B8
:103BF000FCF7F2FA781C03F0E6F92920FCF7ECFA5E
:103C000001352020FCF7E8FA2020FCF7E5FA013422
:103C1000854B1B5D612B00D1ADE00135072DDAD856
:103C2000A0190004000C03F0CEF93A20FCF7D4FAF6
:103C3000305DFFF7F5FB335D1A00683A0A2ACFD9E9
:103C4000652B1AD0642B2ED0662B4CD0672B57D007
:103C5000622BD6D12220FCF7BFFA734B1B195B787D
:103C60009B46A31C98465B46002B7DD06E4B43447D
:103C700099465C460F239A466BE001342820FCF7F6
:103C8000ABFA6A4B1B68102B08D0674B185DFCF72A
:103C9000D9FE2920FCF7A0FA0135B2E7624B185D86
:103CA00003F0C7F9F5E76048021993781B045178CF
:103CB00009060B43D7783F020434025D13431F43C8
:103CC0002820FCF789FA594B1B68102B07D03800C5
:103CD000FCF7B8FE2920FCF77FFA013591E73800A0
:103CE00003F0A7F9F6E701342820FCF775FA4E4BEC
:103CF000185DFFF7BBFB2920FCF76EFA013580E762
:103D000001342820FCF768FA474B1F5D3800FFF7A5
:103D1000ADFB3F01083743483F184020FCF75CFAF1
:103D20003804000C03F085F92920FCF755FA013519
:103D300067E75C20FCF750FA3809FCF743FB504674
:103D40003840FCF73FFB013C01239C46E144002C3A
:103D500009D04B461F783B00203B5E2BE9D838004A
:103D6000FCF73AFAEFE7D8444446013C2220FCF73E
:103D700033FA033545E72C4820180004000C03F003
:103D800022F93A20FCF728FA3B20FCF725FA244BCD
:103D90001A681201234B9B18DA68C0231B051A42CC
:103DA00009D10D20FCF718FA11B0F0BCBB46B246A1
:103DB000A946A046F0BD02A802F079FE1B4B1B6885
:103DC000102B18D0164B1A681201164B9B189868C6
:103DD00002F09FFE2020FCF7FFF94020FCF7FCF9E1
:103DE0000F4B1868000108300E4BC0180004000C7F
:103DF00003F01FF9D5E70A4B1A681201094B9B180B
:103E0000986803F016F9E5E7206B0008346B0008AA
:103E1000486B00089C14002094140020F01400202B
:103E2000CC1400200808002008020020AC14002058
:103E3000134B1B68134A1360134A1268120113498B
:103E40005218BE20C000844661448A420AD21049FA
:103E50000139891A8908013189005118002001C2ED
:103E60008A42FCD10B4A934209D80B4A9B180B4952
:103E70008C4662440021197001339342FBD1704794
:103E800000150020FC140020DC140020080800208D
:103E9000F80D0020FE05000008020020FF050000CC
:103EA00010B5164B1A68164B1A60FEF797F9FEF715
:103EB000DFFA00280DD0114B1A68114B1A60114B14
:103EC0001B68032B0BD8104A802311680B43136027
:103ED00004E00D4A212311680B43136010BD0B4A07
:103EE00013600B4A1B0100219954D318DB681B0592
:103EF0001B0D084A1360FFF79BFFEFE79C1400209F
:103F000094140020CC140020F0140020DC140020B5
:083F1000080800200015002044
:103F180010B50023204A1360204A1360204A13700A
:103F2800204A1360204A1360204A01211160204A68
:103F38001360204B1A68204B1A60204A002311781E
:103F4800002903D0013310325F2BF8D11C4A1360CB
:103F58001C4A1D4BD35C612B1CD01B4B1100013B31
:103F6800CA5C612A02D0002BF9D102E0002B00D0F4
:103F78000133164A1360FFF757FF154A154B1A60AD
:103F880000231360144A0F491160144A1360FDF7A7
:103F980073FC10BD0C4BEBE7F8140020F414002060
:103FA8009F15002008150020E0140020F4010020CF
:103FB800A8140020D8140020AC1400200808002001
:103FC800DC14002008020020FF0500000015002076
:103FD800C0130020C8140020EC140020F0140020A6
:103FE80030B5B9B036AAA04B196836919988918036
:103FF8009B79937134AA9D4B196834919988918063
:104008009B79937131AA9A4B03CB03C211001A888A
:104018000A809B788B702EAA964B13CB13C22BAABF
:10402800954B03CB03C211001A880A809B788B70CA
:1040380027AA924B13CB13C21B88138022A9904B3B
:104048000A0013CB13C203CB03C21CA98D4B0A0071
:1040580013CB13C203CB03C21B78137018AA8A4B65
:1040680013CB13C21B68136014AA884B13CB13C25B
:104078001B8813800FAA864B13CB13C211001A6832
:104088000A609B888B8009A9824B0A0013CB13C254
:1040980003CB03C21B78137005AA7F4B13CB13C243
:1040A8001B78137001AA7D4B13CB13C21B88138096
:1040B8007B4B1A687B4B40339A4200D280E07A49A6
:1040C8000423086803430B60764B0C339A4204D2EE
:1040D800754A042311680B431360744B1B68002B4B
:1040E8000FD0734B1968734B09010022CA545B182F
:1040F8005A709A70DA701A715A719A71DA719A60F4
:10410800DA606A4B00221A606B4B1B68002B0ED0DA
:104118000024694D2020FCF75BF801342B68A3428A
:10412800F8D85E20FCF754F80D20FCF751F836A8B3
:1041380002F0B9FC5C4C206802F041FF3D20FCF71E
:1041480047F82368DB075ED4574B1B689B075ED490
:10415800554B1B685B075ED4534B1B681B075ED42B
:10416800514B1B685B065ED44F4B1B689B065ED4A5
:104178004D4B1B681B065ED44B4B1B68DB055ED49E
:10418800494B1B689B055ED4474B1B685B055ED497
:10419800454B1B681B055ED434A802F084FC464BD3
:1041A8001868FCF74BFC2920FCF712F8FFF7B0FE63
:1041B8000D20FCF70DF8414B00221A6039B030BDD4
:1041C800384B0C339A4200D282E7374B1B68002BDE
:1041D80000D082E7354B1B68002B40D1384B1B6859
:1041E800012BE5D02020FBF7F3FF6F20FBF7F0FF52
:1041F8006B20FBF7EDFF334B1B68102BD8D1482001
:10420800FBF7E6FFD4E731A802F04DFC9CE72EA8A7
:1042180002F049FC9CE72BA802F045FC9CE727A884
:1042280002F041FC9CE722A802F03DFC9CE71CA898
:1042380002F039FC9CE718A802F035FC9CE70FA8AF
:1042480002F031FC9CE714A802F02DFC9CE709A8B9
:1042580002F029FC9CE705A802F025FC9CE701A8D0
:1042680002F021FCA4E7C0468C6B0008946B0008A0
:104278009C6B0008A86B0008B46B0008C06B0008B2
:10428800D06B0008E46B0008FC6B00080C6C00089D
:104298001C6C0008306C0008486C0008586C00085A
:1042A800C014002010140020F0140020F414002082
:1042B800DC140020080800209414002008150020B1
:0842C800F8140020AC140020E2
:1042D00010B50023134A13600A2213490A601349D8
:1042E0000A60134A01211160124A1360124B3122F5
:1042F00056240021C02000051C705A709970D860A7
:10430000996010330132D2B2352AF5D10B4B313AD4
:104310001A60002308493C328B54094A1360FFF7A6
:10432000FBFD10BD6C150020D8140020AC1400203B
:10433000F40100201015002008080020DC140020E3
:044340000015002044
:1043440070B5164C164D2B682360FDF745FF2B689E
:104354002360144B1D68013D28006B1C17D02D01F0
:10436400114BED18114E10E08B420BD1002913D0E4
:104374000132A95C935D1C00613C192CF4D8203BEC
:10438400DBB2F1E7103D013804D30022F1E701204C
:10439400404201E00120404270BDC0469414002018
:1043A4009C140020DC140020080800207013002056
:1043B40010B5FFF7C5FF0400431C0DD002011D4BCF
:1043C4009B18DA68C0231B051A420BD01A4A8023B3
:1043D40011680B43136010BD174A212311680B4366
:1043E4001360F8E7FFF7ACFF431C11D00201114B37
:1043F4009B18DA68C0231B051A420FD1844213D9D3
:104404000C4B24011C19A268000118188260E2E711
:10441400094A212311680B431360DCE7064A802311
:1044240011680B431360D6E7034A802311680B43DA
:0C4434001360D0E708080020F0140020FE
:1044400010B5FFF77FFF431C0FD003010D4AD218B0
:10445000D3681B051B0D0C495B1892689A420AD35E
:104460000001084A1018836010BD084A2123116812
:104470000B431360F8E7054A802311680B43136070
:10448000F2E7C0460808002008020020F0140020CF
:10449000F8B506000D490A68571C0F6054783F199B
:1044A000002C10D00D0005E05878FBF795FE013C7C
:1044B000002C08D02B685A1C2A60012EF4D05878A2
:1044C000FBF756FFF3E7014B1F60F8BDEC1400202B
:1044D000074B1A68511C196051780902901C18602A
:1044E00092781143802292050A431A607047C046B1
:0444F000EC140020A8
:1044F40010B5084B1B681B68002B08D0064A1368CC
:1045040002331360034A1368043B136010BDFFF7C2
:0C451400DDFFF7E7C0140020EC140020CD
:1045200010B5094B1B68191F1A680B689A4208D10D
:10453000064A136802331360034A1368043B13608E
:1045400010BDFFF7C5FFF7E7C0140020EC140020F2
:1045500010B5094B1B68191F1A680B689A4208DDD1
:10456000064A136802331360034A1368043B13605E
:1045700010BDFFF7ADFFF7E7C0140020EC140020DA
:1045800010B5094B1B68191F1A680B689A4208DAA4
:10459000064A136802331360034A1368043B13602E
:1045A00010BDFFF795FFF7E7C0140020EC140020C2
:1045B00010B584B001A8214B020012CB12C21B8897
:1045C000138002F074FA1E4C2068FCF73BFA236853
:1045D0001F2B15D00B2B1DD0194B1B68132B20D074
:1045E000174B1B68262B20D0154B1B68392B20D06E
:1045F0003020FBF7F1FD3020FBF7EEFD04B010BDDD
:104600003220FBF7E9FD3520FBF7E6FD3020FBF714
:10461000E3FDF3E73520FBF7DFFD3220FBF7DCFDA0
:10462000DAE73220FBF7D8FDDAE73420FBF7D4FDD8
:10463000DAE73620FBF7D0FDDAE7C046706C0008F9
:0446400088150020B9
:1046440070B59CB0674B1A681A929A8869466C20B8
:1046540009180A809B796A466E215218137018ADA6
:10466400614B2A0003CB03C2604B1A6816929A88E6
:1046740069465C2009180A809B796A465E215218B3
:10468400137012AC5A4B220043CB43C21B781370F5
:10469400584B1A6810929A8810AB9A80564B1A6835
:1046A4000E929A880EAB9A800AAA544B43CB43C20B
:1046B4001B68136007AA524B43CB43C203AA514B56
:1046C40043CB43C21B6813606A464F4B03CB03C200
:1046D4001B8813804420FBF77DFD6120FBF77AFDE6
:1046E4007420FBF777FD6120FBF774FD1AA802F034
:1046F400DCF946480C3002F064FC280002F0D5F9DD
:104704001AA802F0D2F9424802F05BFC200002F041
:10471400CCF9404802F055FC16A802F0C6F93E4810
:1047240002F04FFC0D20FBF755FD3C4B1B68002BA2
:1047340010D110A802F0B9F90AA802F0B6F907A836
:1047440002F0B3F9364B1B680024002B06D0324E1E
:10475400334D3BE00EA802F0A8F9EDE76E20FBF71D
:1047640039FD6F20FBF736FD6E20FBF733FD652026
:10477400FBF730FD0D20FBF72DFD03A802F095F9A2
:10478400284B18683030C0B2FBF724FD2020FBF71B
:1047940021FD2020FBF71EFDFFF708FF684602F00D
:1047A40084F9214B1868002818D16130FBF712FDF9
:1047B4006C20FBF70FFD6C20FBF70CFD0D20FBF7C5
:1047C40009FD1CB070BDFBF705FD01342B68013BEE
:1047D4001B01F318185D0028F5D1CBE7FCF730F97D
:1047E400ECE7C046846C00088C6C0008946C0008EC
:1047F4009C6C0008AC6C0008B46C0008BC6C00082D
:10480400CC6C0008D86C0008E86C00081014002078
:10481400C013002008020020080800206C150020A6
:0C482400101500206415002084150020F1
:1048300030B58BB003A8124B020032CB32C232CB60
:1048400032C21B8813806A460E4B32CB32C202F052
:104850002EF9FCF70DFB0028FBD0FF231840592848
:1048600008D0684602F023F90D20FBF7B5FC0020C4
:104870000BB030BD0D20FBF7AFFC0120F8E7C046C0
:08488000D0620008EC620008A0
:10488800F0B591B0040001A9334B0A0023CB23C231
:1048980023CB23C223CB23C203CB03C22F4D304EDD
:1048A80033682B60FDF796FC33682B60FDF732FD0B
:1048B800051E08D02B4A802311680B43136000257E
:1048C800280011B0F0BDFDF793FD002804D10CA815
:1048D80001002A00244F0EE001A802F0E4F8FFF7D7
:1048E800A3FF0028F3D10225EAE7002B12D0072AFC
:1048F8000AD001320131D35D0B701E00613E192EC2
:10490800F3D8203B0B70F2E7164A022311680B43D9
:104918001360D5E70CAB1B78002B0CD0134A126838
:10492800120113495218535501354378002B02D010
:104938000130072DF7D10D4B1A6812010C4B9B184B
:104948005D1900226A700B4A10680B4A82189A6037
:104958002043D8600125B3E7F862000894140020CA
:104968009C140020F014002070130020DC14002098
:0C497800080800200015002008020020A4
:1049840070B5C0200005FFF77DFF00280DD00A4C4C
:1049940022680A4803681D010949491915688D6090
:1049A400043A22600133036070BD064A0123116892
:1049B4000B431360F8E7C046C0140020DC14002049
:0849C40008080020F014002097
:1049CC0010B50020FFF75AFF002808D0022807D0A6
:1049DC00074B1A68074B1A60074B01221A6010BD6F
:1049EC00064B1B681B01064A00219954F7E7C04689
:1049FC0000150020FC140020F4140020DC1400200E
:044A0C000808002076
:104A100010B590B008A9284B0A0013CB13C213CBD2
:104A200013C203CB03C201A9244B0A0013CB13C248
:104A300013CB13C21B681360214A13681C68043B24
:104A40001360962C1ED0112C29D0192C03D11324BD
:104A50000B2C1BD002E0312C15D11F24132C15D0A8
:104A60001F2C13D0262C11D0392C0FD0602C0DD038
:104A700001A802F01CF8134A8023DB0011680B43E5
:104A800013600AE06024382C0AD1262408A802F01A
:104A90000EF8FFF7CDFE002806D110B010BD0B2494
:104AA000572CD5D13924F1E7074B1C60074B1C600C
:104AB000FBF71EFBF1E7C0462463000844630008CF
:104AC000C0140020F0140020881500205C15002080
:104AD00010B592B00AA93A4B0A0013CB13C213CBFC
:104AE00013C203CB03C201A9364B0A0013CB13C276
:104AF00013CB13C203CB03C21B881380324A136843
:104B00001C68191F1160314A1268A24220D0304A35
:104B10001268002A14D0043B1B68042B1AD8A31E69
:104B2000022293431DD0012C26D0032C34D0294BD4
:104B30001B68294A12689A4229D1244B1C6007E05D
:104B4000264A802311680B431360204B00221A6011
:104B500012B010BD214A8023DB0011680B431360A3
:104B6000F6E70AA801F0A3FF0D20FBF735FBFFF7DE
:104B70005FFE0028D7D1EBE701A801F098FF0D20D8
:104B8000FBF72AFBFFF754FE0028D0D1E0E7124ADA
:104B90001360FBF7ADFAD0E701A801F088FF0D2004
:104BA000FBF71AFBFFF744FE0028D1D00A4B094A55
:104BB000196811601F221A60FBF79AFABDE7C04618
:104BC000006D0008206D0008C0140020641500204E
:104BD000881400205C15002088150020F0140020A7
:104BE00030B585B0174B1A6802929A8869468A8157
:104BF0009B798B73144B1A6800929A888A809B79F0
:104C00008B71FCF7D3FA114C23681D6802A801F0E0
:104C10004EFFFDF775F82020FBF7DEFA23681C68CD
:104C2000684601F044FFFDF76BF82020FBF7D4FA4B
:104C3000FFF7FEFD002803D0054B1D60054B1C60EF
:104C400005B030BD046F00080C6F0008C0140020D0
:084C500014150020701500206E
:104C580030B589B001A80B4B020032CB32C232CB3F
:104C680032C21B68136001F01EFFFFF7DDFD00284C
:104C780001D109B030BDFBF7CDFC034B01221A600E
:0C4C8800F7E7C046606300086C150020D0
:104C940010B58CB006A91E4B0A0013CB13C203CB6C
:104CA40003C21B78137069461A4B0A0013CB13C254
:104CB40003CB03C21B781370174A13681968043BAB
:104CC400136001290ED8002914D1684601F0EDFEC5
:104CD400FFF7ACFD00280BD0104B00221A60FFF741
:104CE400F5FA05E00E4A8023DB0011680B431360DC
:104CF4000CB010BD06A801F0D8FEFFF797FD002800
:104D0400F6D0064B01221A600120FBF785FAEFE783
:104D1400946E0008AC6E0008C01400206C150020CE
:044D2400F014002067
:104D2800074B1B68002B09D0054B00221A60054A67
:104D38001368191D1160044A12685A607047C0460A
:0C4D480008150020C014002004150020F5
:104D540010B5214B1A68214B1A60FDF73DFAFDF797
:104D640085FB002821D01C4B1A681C4B1A601C4B75
:104D74001A6812011B4B9B18DA68C0231B051A42E0
:104D840019D0194B1B78002B1BD1184B1B68002B17
:104D94001AD117480368124A11680901114A5218B6
:104DA40019689160043B036004E0124AA02311686F
:104DB4000B43136010BD0F4A802311680B4313602B
:104DC400F8E7FFF7AFFFE0E76720FDF7B9FB044B17
:104DD4001868FDF7B5FBEDE79C140020941400203F
:104DE400CC140020080800209F150020F414002093
:084DF400C0140020F01400209F
:104DFC00F0B5C64600B588B069462B4B0A0013CBFC
:104E0C0013C213CB13C203CB03C2284B1B78002B4A
:104E1C0014D1274A13688024A40519680C43043B59
:104E2C001360244B9C420CD9234A8023DB0011686D
:104E3C000B43136008B080BCB846F0BDFFF76EFFA3
:104E4C00E7E70D20FBF7C2F9684601F02AFE2000C7
:104E5C0002F0B3F8270080370F25032398460FE0A4
:104E6C000D20FBF7B3F9200002F0A7F83A20FBF76E
:104E7C00ADF9300001F02BFE00250134BC420ED000
:104E8C0026780135102DEBD0300001F020FE434682
:104E9C002B40032BF1D17C20FBF798F9EDE70D208B
:104EAC00FBF794F9C6E7C0467C6300089F15002009
:0C4EBC00C0140020807F0020F0140020B3
:104EC80082B03A4B1A6801210A431A605A68384876
:104ED80002405A601A68374802401A601A68364811
:104EE80002401A605A68354802405A60DA6A0F2050
:104EF8008243DA621A6B324802401A635A6B8A4359
:104F08005A6300229A600092019219688022520224
:104F18000A431A60190080229202A020C0010B687F
:104F280013400193009B01330093019B002B02D196
:104F3800009B8342F3D11D4B1B689B0306D50123BD
:104F48000193019B012B04D002B070470023019309
:104F5800F7E71C4B11221A60144B5A685A605A68BA
:104F68005A605A6818490A405A6059688822520398
:104F78000A435A601968802252040A431A601900C9
:104F8800802292040B681342FCD0084B5A68032114
:104F98008A435A605A6801390A435A6019000C2238
:104FA8004B681340082BFBD1CEE7C04600100240E7
:104FB8000CB8FFF8FFFFF6FEFFFFFBFFFFFFC0FF87
:0C4FC800ACFEFFFF00200240FF7FC0FF96
:104FD4000E4B00221A609022D20513680C490B4034
:104FE40013600C4A802380210906D150BFF34F8FF0
:104FF400BFF36F8F084B1969802212040A431A61A8
:10500400DA6906490A40DA617047C046881400200C
:10501400FFFFC3FF00E100E000100240FFFF7FFF3D
:105024004C4B80221A6000224B4B1A604B49086893
:1050340080231B0203430B60494B1A601B68494AD7
:105044009A1849490A6049490A604949581849491E
:105054000860494958184949086049495818494954
:105064000860494958184949086049495818494944
:105074000860494958184949086049498C466344BD
:1050840048490B60484B1B68002B06D113001833AA
:1050940046490B60464902330B6040231380354B6D
:1050A4001B6800221A80354B1B6880211980354B00
:1050B4001B6840491980354B1B68802040001880CC
:1050C400344B1B681A80284B1B689881DA810130A5
:1050D400FF3018825A82314B1B681880314B1B6891
:1050E4001980314B1B68002B0BD1304B1B68C0213E
:1050F400890019802E4B1B681A801B4B1B689983EF
:10510400DA832D4B2D4A1A802D4B2E4A1A802E4BB2
:105114002E4A1A80244B1B68002B02D12C4B2D4A9B
:105124001A802D4BBF2212021A6000232B4A1360EF
:105134002B4A13602B4A2C490A602C490A602C4ADA
:105144002C490A602C490A602C4A13702C4A1370AB
:105154007047C0464C5C004090140020585C0040EE
:10516400505C0040006000408C1400204C1500206E
:1051740002600040381500200460004050150020F3
:10518400066000403C1500200860004048150020DF
:105194000A600040341500201460004044150020CB
:1051A40016600040301500208414002040150020B3
:1051B4002C1500200084FFFF005C0040203200001A
:1051C400045C004031300000085C004032300000D4
:1051D4000C5C004033360000405C0040701400203A
:1051E40088140020F80D0020201500201C15002034
:1051F400C41100202815002024150020F9100020D7
:0452040092150020DF
:1052080070B5204CE36980252D042B43E361FAF740
:105218005FFF23691D432561FAF75AFF236B80223C
:10522800134323632369184A134023619022D2054C
:10523800136816490B401360154B0021154A198055
:1052480002339342FBD1144B0021144A19800233D4
:105258009342FBD1124A116880231B020B4313604F
:10526800104C01232360C820FBF7C6F900232360F4
:10527800094A1360FFF7D2FE0B4B802212061A6010
:1052880070BDC04600100240FFFF7FFFFFFFC3FF55
:10529800005C0040205C0040445C0040605C0040D2
:0C52A800585C0040405C004000E100E069
:1052B40070B582B0284B1B68402B45D9274B1B681F
:1052C40040221A80244A1368403B1360234B1B6816
:1052D4001B88002B16D0224C002122481F4D036846
:1052E4001E785A1C02605A78023303601302334357
:1052F40023800234013189B22B681B8801335B108F
:105304009942ECDB184B1B881B0604D5164A1388FC
:1053140016490B401380164B1B68164A1A80124B11
:105324001B889BB26A46D380D3889B0602D40E4B5B
:10533400114A1A806B4606331B88DB0602D40A4BDB
:105344000E4A1A8002B070BD034B1968034A1268F2
:10535400118000221A60B9E770140020381500206B
:10536400406000407C140020005C00400F8FFFFF71
:105374003C1500200084FFFFA082FFFF9082FFFF06
:1053840082B0174B1B6800221A80164B1B881B0621
:1053940004D5144A138814490B401380104B1B681E
:1053A40000221A800F4B1B889BB26A46D380D38895
:1053B4009B0602D40B4B0D4A1A806B4606331B889E
:1053C400DB0602D4074B0A4A1A806B4606331B8855
:1053D4005B0402D5034B074A1A8002B07047C046EB
:1053E40038150020005C00400F8FFFFFA082FFFFF4
:0853F4009082FFFF80C2FFFF61
:1053FC0000B583B01C4A13881C490B4013801C4B0E
:10540C001B68052B1DD01B4B1B68002B29D1164B81
:10541C001B881BB2002B1EDB134B1B889BB26A46EE
:10542C00D380D3889B0402D40F4B134A1A806B464B
:10543C0006331B88DB0402D40B4B104A1A8003B0D2
:10544C0000BD0F4B1B68802213430E4A1360084BA0
:10545C0000221A60D7E7044A13880B490B401380CB
:10546C00DAE7FFF721FFEAE7005C00400F8FFFFF50
:10547C00741400207014002080A2FFFF8092FFFFA4
:0C548C00901400204C5C00408F0F0000CA
:1054980082B0134B1A8813490A401A801B881B06CE
:1054A80004D50F4A138810490B4013800C4B1B88F6
:1054B8009BB26A46D380D388DB0602D4084B0B4ADA
:1054C8001A806B46DA8806331B889B0402D4044B87
:1054D800074A1A806B4606331B8802B07047C046DD
:1054E800005C00408F0F00000F8FFFFF9082FFFFCE
:0454F80080A2FFFF90
:1054FC0030B587B0C54B1B881B0500D4D0E1C34A1F
:10550C001388C3490B401380C24B1B78C2490B70E4
:10551C00C24B1A78C24B1A70C24B1A88C24B1A80F3
:10552C001A88120AC14802701B88DBB2C04A137079
:10553C00C04B1A88C04B1A80C04B1A88C04B1A80BB
:10554C00C04B00221A60C04B1B68C04A1A800B78F3
:10555C00212B31D0B04B1B78DBB2A12B62D0AE4BE0
:10556C001A7861231A4206D0AB4B1B786122134088
:10557C00012B00D046E1A54A1388A5490B401380A6
:10558C00A74B1A78D3B2062A00D17DE0062B66D839
:10559C00002B70D0052B00D025E1AD4B00221A60FA
:1055AC00FFF7EAFEA04B1B887F221340A94A136029
:1055BC00A44B05221A607FE1994B1B78202B0BD052
:1055CC00974B1B78222B2AD1904A138890490B4079
:1055DC001380FFF7D1FE6FE18C4B1B889BB2162218
:1055EC006A44138013889B0402D4884B9A4A1A800D
:1055FC0016236B441B88DB0402D4844B974A1A8015
:10560C0016236B441B885B0403D5804BA0229200AD
:10561C001A807E4A13881BB2002BFBDB4CE1FFF790
:10562C0035FF49E17E4B1B78212B98D1774A1388A3
:10563C0077490B401380864A07231360804B1B88E5
:10564C009BB21268934204D27D4B1B889BB2804A5A
:10565C001360834B834A1A60FFF726FE2CE1092B5B
:10566C0000D0C0E07A4B00221A60FFF785FE7E4B1B
:10567C00FF221A6020E1764B02221A60784B7B4A9B
:10568C001A60FFF711FE17E1684B1B78012B28D02D
:10569C00664B1B78022B5ED0644B1B78032B00D01F
:1056AC009EE0634B1B78012B73D0614B1B78022B54
:1056BC0000D180E05E4B1B78002B00D08DE0644A5B
:1056CC00043313605E4B1B889BB21268934204D266
:1056DC005B4B1B889BB25E4A1360614B644A1A6039
:1056EC0028E05B4B12221A60624B1B68012B24D002
:1056FC00614D5B4B1D60614B1C68614A01239442F8
:10570C001DD0681E6A46D11CC25CCA540133132BCF
:10571C00FAD101AB1C72240A5C725A4B9D4215D013
:10572C00594B1A7801AB9A72574A1268120ADA72FC
:10573C004B4A1360FFF7B8FDBEE0524DD9E7534B0F
:10574C00514A12689A42F5D00123DAE74E4B1A6897
:10575C000332D2B2E6E7474B1B68012B12D03C4B0D
:10576C0043221A603E4B4A4A1A60354B1B889BB247
:10577C00374A12689342DDD2314B1B889BB2344AB4
:10578C001360D7E7324B65221A60354B414A1A60D9
:10579C00EBE72F4A17331360294B1B889BB2126817
:1057AC00934204D2264B1B889BB2294A13602C4B84
:1057BC00394A1A60BEE7264A10331360204B1B8807
:1057CC009BB21268934204D21D4B1B889BB2204A99
:1057DC001360234B314A1A60ACE7FFF757FE6BE0BE
:1057EC00FFF754FE68E00C4B1B78002B02D0FFF740
:1057FC004DFE61E0054A138805490B401380FFF705
:10580C00BBFD59E0FFF742FE56E0C046005C00408D
:10581C008F0F0000806000409315002081600040D5
:10582C009415002082600040FA1000209C15002086
:10583C009D1500208460004090150020866000407B
:10584C008A120020741400203C1500200084FFFFF5
:10585C00701400209014002080A2FFFF8092FFFFA4
:10586C007C140020586F000888140020706D00080C
:10587C007869000884140020506D0008141500206D
:10588C0083040000A06D0008701500204057000034
:10589C00146F0008606F00087C690008806D0008B8
:1058AC00094B1B889BB216226A44138013881BB2C7
:1058BC00002B03DBFFF760FD07B030BD1388034AF4
:1058CC001340014A1380F5E7005C00408F0F000085
:1058DC00F0B5DE4657464E464546E0B583B03C4BE8
:1058EC001B881B0604D53A4A13883A490B4013808F
:1058FC00394C0022394FB846394B9C46BA46B9460A
:10590C0033E05346374E1E6044E001AB1B882B80BE
:10591C005A46354B1B681A802D4B1B889BB26A4626
:10592C00D380D3889B0602D4294B304A1A806B460D
:10593C0006331B88DB0602D4254B2D4A1A8003B094
:10594C00F0BCBB46B246A946A046F0BD254B234948
:10595C000B600232D2B26B46598801AB1B8809022C
:10596C000B432B80402AD4D00234A51E3B6821491E
:10597C0008688342CDD0694600264E8019788B4644
:10598C0001A95E460E80013341460B6061460968F1
:10599C008B42B6D0531CDBB29B46402BB5D04B464A
:1059AC001B6883420AD01878834668465E46468058
:1059BC0001339942CAD009490B60CAE76B465A8831
:1059CC0001AB1B88120213432B805A46CCE7C0460E
:1059DC00045C00400F8FFFFF026100401C1500208B
:1059EC00F8010020F80D002034150020A180FFFFE5
:0859FC009180FFFF201500203F
:105A040082B0114B1B881B0604D50F4A13880F491B
:105A14000B4013800E4B1B6800221A800A4B1B8814
:105A24009BB26A46D380D3889B0602D4064B094AAC
:105A34001A806B4606331B88DB0602D4024B064AE7
:105A44001A8002B07047C0460C5C00400F8FFFFF05
:0C5A54002C150020A386FFFF9386FFFFA7
:105A600010B5204B1B68002B34D01F4B1868002842
:105A70002FD01E4B1A681E4B1B689A4230D0511C07
:105A80001A48016014781B4A1268914225D0174ABF
:105A90001268991A934201D2C433991A164B1B68A3
:105AA000002B11D07D290FD8134B00221A60134B05
:105AB0001B889AB29B0402D4104B11491980D3045D
:105AC00002D40E4B0F4A1A80FAF7FAFA802000022D
:105AD000204310BDFAF726FDC7E70B490160D6E762
:105AE0000020F6E768150020881400202415002007
:105AF00028150020FC01002078140020085C0040DC
:0C5B000082A0FFFF8290FFFFC411002074
:105B0C0070B5634B19684A1C1A60012800D1B9E0C2
:105B1C000A788B1C5E4C2360022800D1B4E04D78CF
:105B2C00CB1C2360032800D1B0E08E780B1D2360C2
:105B3C000438C0B2931E0D2B00D9A4E0052A32D034
:105B4C000F2A30D013000C3B012B3DD90423140039
:105B5C009C43022C5AD0C978072A7AD84D4B002284
:105B6C001A704D4B1A68541C1C6015701A684B4BFC
:105B7C001B689A4269D0484B1A68541C1C601670FA
:105B8C001A68464B1B689A4278D0434B1A68541CCF
:105B9C001C6011701A68414B1B689A4273D13E4BC2
:105BAC003F4A1A606FE03B4B00221A703A4B1A685E
:105BBC00511C196015701A68384B1B689A4262D1D7
:105BCC00354B374A1A605EE0324B1B78AB420BD038
:105BDC00314B1A68511C196015701A682F4B1B68D1
:105BEC009A420FD02B4B1D702B4B1A68511C19600D
:105BFC0016701A68294B1B689A4244D1264B284AC6
:105C0C001A6040E0244B264A1A60EBE7214B002235
:105C1C001A70214B1A68511C196015701A681F4BA9
:105C2C001B689A420DD01C4B1A68511C19601670D7
:105C3C001A681A4B1B689A4225D1174B184A1A60DE
:105C4C0021E0154B164A1A60EDE7134B144A1A6003
:105C5C0091E7104B1B78AB428DD00F4B1A68541C3C
:105C6C001C6015701A680D4B1B689A4202D0094BC8
:105C7C001D7080E7084B0A4A1A60F8E7064B084A81
:105C8C001A6082E7002070BD0020FCE70020FAE7D4
:105C9C00801400209215002028150020FC01002003
:045CAC00C4110020FF
:105CB00070B582B0404B1B881BB2002B11DB3F4BF1
:105CC0003F4A1A603F4B1B6818783F4B1B685A00CD
:105CD000D21890423FD940283DD83C4D374C260041
:105CE00025E0354A13883A490B401380E7E7FFF770
:105CF0000DFF14E0374B02221A600BE0364B1A6896
:105D0000511C19603168097811701A68334B1B688F
:105D10009A421CD02368013323600138C0B22A4B59
:105D20001B685A00D218904215D9402813D8012B6D
:105D3000DDD02B68022BE1D0204B1B681B78022B97
:105D4000D8D0042BDAD1234B04221A60E2E7224B8D
:105D5000234A1A60DEE7234B1A681F4B1B689A42DE
:105D600020D99B1AC4339BB201AA13801E4B002278
:105D70001A6001AB1B889BB27E2B18D80E4B1B8878
:105D80009BB26A46D380D3889B0402D40A4B174A3D
:105D90001A806B4606331B88DB040BD4064B144A6F
:105DA0001A8007E09B1A9BB201AA1380DEE70E4B14
:105DB000FF321A6002B070BD085C00408014002001
:105DC000006200403015002084140020641500207B
:105DD0008F0F0000A414002028150020FC010020D3
:105DE000C4110020241500207814002082A0FFFF99
:045DF0008290FFFF9F
:105DF40000B585B0234B1A6801921B681B0429D592
:105E0400019A0F2313400393019A10231340029322
:105E1400039B012B0BD0039B022B0BD0039B002B6A
:105E24000ED1029B002B08D1FFF7E6FA1DE0FFF725
:105E340053FD1AE0FFF73AFF17E0FFF75DFB14E0AC
:105E4400039B032B11D1104B1B68002B0DD1FFF7C3
:105E5400D7FD0AE00B4B1B685B0508D4094B1B6894
:105E64001B050AD5074B094A1A6005B000BDFFF7A8
:105E7400D7F8044B064A1A60F7E7024B054A1A6042
:105E8400F3E7C046445C004084140020FFF7FFFFA2
:085E9400FFFBFFFF7F8000000F
:105E9C0070B5134B1B68002B21D0124B1A68511C88
:105EAC00196010701A68104B1B689A4204D00F4E80
:105EBC000C4DAC24A4000AE00A4B0D4A1A60F6E71C
:105ECC00C02189008C466344991AA14207D9FAF77C
:105EDC0023FB32682B68991A9A42F6D9F0E770BD09
:105EEC008814002020150020F80100201C1500202B
:045EFC00F80D00207D
:105F000000B5C54A13780133DBB2137042B2002AE0
:105F100023DBC24B1B78002B00D1A2E0C04B1B78C7
:105F20000F2219009143BF4A1278002A00D0BCE02A
:105F3000BD4A1070BD4A0020107002221800904324
:105F40000200F12800D195E01F229343C02B00D11D
:105F50009DE0B44BFF221A708BE0F72800D139E1A5
:105F6000AD4B01221A70F0281BD0AD4B1870F328EE
:105F700062D903000C33DBB2012B68D9FD2866D04F
:105F8000AB4B05221A700023A74A1370A74A13705F
:105F9000A24A1370A34A1370A64A1370A64A13703C
:105FA000D1E09F4BEF321A709C4B0F321A700023D6
:105FB0009C4A13709F4A13709F4A137059E09C4B80
:105FC00005221A70964BF2321A700023964A13700B
:105FD000964A1370914A1370924A1370954A13703F
:105FE000954B1B78002B03D0934B00221A70AAE02C
:105FF0000023894A1370904A13703AE08C4B0622B2
:106000001A70894B1978864A1170F7221A7000238A
:10601000864A1370814A1370824A1370854A13703E
:10602000854A13708FE0844B1B78002B00D0DFE093
:106030007E4BF0321A70E4E0784BFF221A70002396
:10604000784A13707B4A13707B4A137011E0002367
:10605000724A1370734A1370764A1370764A13703B
:1060600007E06D4A13706F4A1370724A1370724AD8
:10607000137000BD6E4BEF3A1A700023674A13701D
:10608000684A13706B4A13706B4A13705BE009091E
:10609000674B1970614BE0321A700023614A13702C
:1060A000644A1370644A13704DE0624A1278002A01
:1060B00034D15E4A1070604A1278002A0FD1F22B58
:1060C00011D0F02B1CD00909594B1970534BFF22EA
:1060D0001A700023534A1370564A137033E0554B1D
:1060E000FF221A70C5E7524B03221A7000234B4A55
:1060F00013704C4A13704F4A13704F4A137022E0CA
:106100004B4B04221A70FF234B4A1370434A1370FF
:106110000023444A1370474A137014E0424A11782E
:106120003F4B1970414B197811701870404B042285
:106130001A70FF23404A1370384A13700023394AFB
:1061400013703C4A13703D4B1B68002B00D190E745
:106150003B4B1A68531C364909781170394A12684A
:106160009A422FD05A1C2E4909781970354B1B685A
:10617000934229D0531C2C4909781170314A126876
:106180009A4223D05A1C2949097819702D4B1B6853
:1061900093421DD02A4B1A6000231F4A1370214AD4
:1061A0001370244A1370224B1B78072B01D8042B41
:1061B00004D11B4B1B78F02B00D85AE7174B002259
:1061C0001A7056E7204BCDE71F4AD3E71E4BD9E79D
:1061D0001D4ADFE7012B00D1F1E6022B00D10DE7CC
:1061E000134B07221A700E4B1B78F02B00D11AE7C5
:1061F0000D4A11780A4B19700C4B19781170F7225F
:106200001A700023054A1370064A1370094A137066
:10621000094A137097E7C046F91000209615002030
:10622000971500209B150020991500209815002037
:10623000951500209A15002089120020881400204E
:0C62400020150020F8010020F80D0020BF
:10624C00074B1B68002B00DBFEE7054A1168802317
:10625C001B060B4313608369023383617047C0468E
:04626C002CED00E035
:1062700043466F72746820666F722053544D3332F8
:106280004630343220762E002028632932303230D6
:106290002D323420572E536368656D6D657274001E
:0862A000202D3E44424720007E
:0862A8004B65726E656C3A0053
:1062B000C83200081E33000878330008783300081D
:1062C00030330008423300085433000866330008B6
:1062D00020636F6E6669726D20772E7570706572BF
:1062E0002063617365202759270000002063616ED9
:0862F00063656C6C656420001D
:1062F800205761726E3A2077696C6C206F766572F0
:1063080072696465204B65726E656C204F5020770A
:0C6318002E73616D65206E616D652000C4
:10632400426175642052617465206368616E6765BB
:106334007320696D6D6564696174656C79212000F1
:10634400656E746572204F4E4C5920464952535421
:0C635400203220444947495453212000C6
:10636000536176652061637475616C20776F726B21
:0C63700020696E20466C617368203F00BD
:10637C00313238205352414D206279746573207349
:10638C0074617274696E672066726F6D203078006C
:10639C0000000000000000000000000000000000F1
:1063AC0000000000000000000000000000000000E1
:1063BC0000000000000000000000000000000000D1
:1063CC0000000000000000000000000000000000C1
:1063DC0000000000000000000000000000000000B1
:1063EC0000000000000000000000000000000000A1
:1063FC000000000000000000000000000000000091
:10640C000000000000000000000000000000000080
:10641C00000000000000000000000000000001006F
:10642C00000005000000000000000000000000005B
:10643C000000000000000000000000000000000050
:10644C000000000000000100000004000000040037
:10645C000000000000000000000000000000000030
:10646C00000001000000000000000000000000001F
:10647C000000000000000000000000000000000010
:10648C000000000000000000000000000000000000
:10649C0000000000000004000000000000000500E7
:1064AC0000000500000005000000040000000400CE
:1064BC0000000400000004000000000000000100C7
:1064CC0000000100000001000000010000000300BA
:1064DC0000000300000003000000030000000300A4
:1064EC000000030000000300000003000000030094
:1064FC000000030000000300000003000000020085
:10650C000000020000000200000002000000020077
:10651C00000001000000010000000800000008005D
:10652C00000008000000080000000800000008003F
:10653C00000008000000080000000800000008002F
:10654C00000008000000080000000800000008001F
:10655C000000080000000800000008000000020015
:10656C00000002000000010000000100000001001A
:10657C000000010000000100000005000000010007
:04658C00000001000A
:106590004552524F5200000044524F50000000003C
:1065A00044555000000000005357415000000000C7
:1065B0004F56455200000000524F540000000000AA
:1065C0002D524F54000000005049434B0000000082
:1065D000524F4C4C00000000494E4A4543540000C5
:1065E0002B00000000000000312B00000000000024
:1065F0002D00000000000000312D00000000000010
:106600004142530000000000534849465400000036
:10661000414E4400000000004F5200000000000006
:10662000584F5200000000004E4F54000000000080
:106630002B2F2D00000000002A00000000000000A9
:106640002F000000000000002A2F000000000000C2
:106650004D4F4400000000002F4D4F44000000004B
:1066600052414E444F4D00003D3D000000000000EF
:10667000213D0000000000003E000000000000007E
:106680003E3D0000000000003C0000000000000053
:10669000553C0000000000003E3D000000000000EE
:1066A000303D000000000000564152434F4E0000B4
:1066B0005245560000000000570000000000000096
:1066C00052000000000000004B45593F0000000050
:1066D0004B45590000000000454D495400000000A2
:1066E0002E000000000000002E4800000000000006
:1066F0002E440000000000002E22000000000000D8
:10670000445A00000000000048580000000000004B
:1067100052583F00000000005258000000000000E6
:1067200054580000000000004E54580000000000C3
:106730005458220000000000584E4F500000000046
:106740004D53000000000000445300000000000012
:10675000544958000000000054494D450000000015
:106760004F480000000000004F4C000000000000F7
:10677000495055000000000049504400000000004E
:10678000495A0000000000005244494E0000000039
:1067900052414443000000002E530000000000005E
:1067A00046530000000000004F505300000000005E
:1067B00055534552000000005345450000000000BD
:1067C0004D454D0000000000535400000000000043
:1067D00052554E00000000004E4F2D44424700002D
:1067E0004445425547000000464F5247455400007B
:1067F00041424F52540000005245504C4143450025
:10680000524553544F5245004946000000000000D5
:1068100043415345000000003C4341534500000004
:106820003E43415345000000454C534500000000E5
:106830005448454E00000000444F00000000000096
:10684000554E54494C0000005748494C4500000043
:10685000414741494E000000464F520000000000F1
:106860004C4F4F50000000004900000000000000A5
:10687000434F4E5449000000425245414B00000036
:106880005A425245414B000052455455524E000069
:106890003A000000000000003B0000000000000083
:1068A000646F535452000000646F494F53545200B8
:1068B000646F4C4954000000646F4C4954384200E6
:1068C000646F56414C554500646F524556000000B8
:1068D000646F494600000000646F43415345000067
:1068E000646F3C4341534500646F3E434153450050
:1068F000646F454C53450000646F444F0000000036
:10690000646F554E54494C00646F5748494C4500DC
:10691000646F414741494E00646F464F520000008A
:10692000646F4C4F4F50000052502D31000000005A
:1069300052502D34000000004155544F4558450039
:1069400042415544000000004348414E4E454C0032
:1069500053504C49540000005649445049440000EB
:106960003F000000000000005341564500000000B9
:086970004C4F414400000000FF
:046978000403090407
:10697C001803430046006F007200740068002D007D
:08698C004D00490044004900E0
:10699400FEE7FEE7FEE7FEE7FEE7FEE7FEE7FEE7CB
:1069A400FEE7FEE7FEE7FEE7FEE7FEE7FEE7FEE7BB
:1069B400FEE7FEE7FEE7FEE7FEE7FEE7FEE7FEE7AB
:1069C400FEE7FEE7FEE7FEE7FEE7FEE7FEE7FEE79B
:1069D400FEE7FEE7FEE7FEE7FEE7FEE7FEE7FEE78B
:1069E400FEE703488546FEF76DFA03E070470000B2
:0469F4000018002067
:1069F80011488546114C20680434004201D0804774
:106A0800F9E70F480F49091A082903DB0022026039
:106A1800043001600C480D49884205D002680430F2
:106A280003B4904703BCF7E700208646EC460020F5
:106A38000021074A9047FEE700180020F070000880
:106A4800A0150020E8160020C96D0008C96D0008CF
:046A5800390C0008ED
:106A5C0004207146084202D1EFF3088001E0EFF305
:0C6A6C0009800149084700004D62000845
:106A78002030204348414E4E454C20616363657089
:106A8800747320414E59204D494449206368616E12
:106A98006E656C20696E2072656365697665642031
:066AA8006D73677320000E
:106AAE0010B5441C0078002806D0F9F78EFB01348F
:0A6ABE00631E18780028F8D110BDFF
:106AC800756E646572666C6F77212000202D2D2D00
:026AD80020009C
:106ADA0010B5040003061B0F18003030392801D9FD
:106AEA0037331800F9F773FB0F20044020003030C9
:106AFA00392800D90730F9F76AFB2020F9F767FB34
:026B0A0010BDBC
:066B0C002849502D3E0057
:0E6B120010B5F9F796FF2020F9F75DFB10BDD6
:106B200063616E277420534545204B65726E656C1A
:106B30004F707300557365724865616465725F5389
:106B400074727563743D0000566172436F6E3A56FD
:066B5000616C75653D005B
:106B56002F280FD90300303BDBB2092B08D90A29AD
:106B66000BD00300413B052B0AD83738C0B270471B
:106B76001800FCE701204042F9E701204042F6E711
:066B860001204042F3E78C
:106B8C004572726F722300002028636F6C20000026
:106B9C00206E6F7420666F756E6400005F53796EA3
:106BAC0074617820457272005F537461636B204589
:106BBC00727200005F436F6D70696C65206F6E6C54
:106BCC00790000005F4E6F20492F4F20436F6D6D91
:106BDC0020416363657373005F496E76616C696411
:106BEC0020436F646520616363657373000000006C
:106BFC005F6F7574206F6620436F6E7465787400D8
:106C0C005F52756E74696D65206F6E6C7900000053
:106C1C005F5468726561642063616E63656C6C655A
:106C2C00640000005F4E756D626572206F75742094
:106C3C006F662052616E6765000000005F446976E4
:106C4C002E6279205A65726F000000002020636F5D
:0A6C5C006D70696C696E672E2E00E2
:0A6C660010B50120FBF765FF10BD1B
:0A6C700042617564526174653D00D5
:0A6C7A0010B50020FBF75BFF10BD12
:106C8400537461636B3D00002052657475726E002D
:106C940020557365723D000020436F64655468722B
:106CA4006561643D00000000456D7074790000006A
:106CB400466C6173680000005F50726F6A656374AC
:106CC400206C6F61646564002020204155544F4559
:106CD40058453D005465726D696E616C5F53706C0C
:0E6CE40069743D0020204D69646943683D00DD
:0E6CF20010B56820FBF725FCFCF755FB10BD24
:106D0000555342205465726D696E616C5F436F6DBF
:106D10002077696C6C20676574206C6F7374210038
:106D20005553415254205465726D696E616C5F43D6
:106D30006F6D2077696C6C20676574206C6F73745D
:026D4000210030
:0E6D420010B56920FBF7FDFBFCF72DFB10BD23
:106D50001201000200000040830440572404000098
:026D6000000130
:0E6D620010B56A20FBF7EDFBFCF71DFB10BD22
:026D7000000021
:0E6D720010B56B20FBF7E5FBFCF715FB10BD21
:106D8000120368006F006D0065006D006100640013
:026D900065009C
:0E6D920010B56E20FBF7D5FBFCF719FB10BD0A
:106DA0001201000200000040830443572404020142
:026DB0000001E0
:0E6DB20010B56F20FBF7C5FBFCF709FB10BD09
:096DC00028566172436F6E3D001C
:0E6DCA0010B57020FBF7B9FBFCF7FDFA10BD09
:106DD800203C2D6E6F742061204B65726E656C20AF
:106DE8004F50206E6F722061206E756D6265720063
:106DF800203C2D696E76616C696420666F72204252
:106E080061636B2D4374726C00000000203C2D52AE
:0D6E1800756E74696D65204572726F7200B1
:0A6E260010B50120FDF731FB10BD8F
:106E300020202841444320696E6974292000000005
:0D6E4000202028414443206F666629200071
:0A6E4E0010B50020FDF71DFB10BD7C
:106E58002064656275672066696E69736865642079
:016E68000029
:106E6A000A0010D00300400800E052008242FCD918
:106E7A00002000E05208934200D39B1A40418A4204
:0A6E8A00F8D119007047002070478E
:106E94004C6F616420466C6173682050726F6A6540
:106EA4006374203F000000004C6F616420456D70E6
:0D6EB40074792050726F6A656374203F008E
:106EC2008446002A05D00B78037001300131013A63
:066ED200F9D16046704793
:106ED800555342206173207669727475616C204342
:106EE8004F4D3D00555342206173204D4944492080
:0B6EF800696E746572666163653D00A1
:0F6F0400564944203D200000504944203D2000C4
:106F14000902430002010080310904000001020259
:106F240000000524001001052401030004240207C5
:106F3400052406000107058303100040090401002D
:106F4400020A000000070581024000000705020252
:036F5400400000FA
:076F580000C2010000000867
:106F600009026500020100803109040000000101EE
:106F700000000924010001090001010904010002C7
:106F80000103000007240100014100062402010161
:106F90000006240202020009240301030102010089
:106FA00009240302040101010009058102400000D7
:106FB0000000052501010309050202400000000050
:056FC00005250101019F
:106FC60010B50400000F16D12001000F17D12002C2
:106FD600000F18D12003000F19D12004000F1AD179
:106FE6002005000F1BD12006000F1CD10F202040CA
:106FF600F9F7E5F910BDF9F7E2F92001000FF9F705
:10700600DEF92002000FF9F7DAF92003000FF9F78D
:10701600D6F92004000FF9F7D2F92005000FF9F789
:0C702600CEF92006000FF9F7CAF9DFE7E9
:1070320010B504003020F9F7CEF87820F9F7CBF834
:087042002000FFF7BFFF10BDA5
:10704A00CA1751408B1A17D0C1174A4004B4484096
:10705A00411A48081A0000E052008242FCD9002076
:10706A0000E05208914200D3891A40419A42F8D16D
:0C707A0004BC5040801A70470020704792
:107086000A000FD00300400800E052008242FCD9FB
:10709600002000E05208934200D39B1A40418A42E6
:0870A600F8D17047002070478B
:1070AE00CA1751408B1A19D0C11706B44840411A5D
:1070BE0048081A0000E052008242FCD9002000E08D
:1070CE005208914200D3891A40419A42F8D10CBC21
:1070DE0053405840C01A5140891A704700207047DB
:1070F0001973000808020020981300002F7300087D
:1071000000000020107100080802000000000000CC
:1071100045110008551100087D110008AD11000847
:10712000C5110008D9110008FD110008211200083E
:1071300061120008C1120008211300083D13000865
:107140004D13000869130008791300089113000813
:10715000D9130008F5130008111400082D140008B5
:107160003D1400084D14000869140008A11400081B
:10717000D9140008111500085115000869150008F8
:1071800089150008BD150008E1150008051600085E
:107190002916000849160008A915000885490008A5
:1071A000554D00086D160008AD160008512A00085C
:1071B0005D1C0008B91B0008B91C0008011D00086F
:1071C000E91E0008676C0008E116000801170008B6
:1071D000AD2C0008492E0008011F0008191F0008E7
:1071E0007B6C000821170008F52E0008252F0008E9
:1071F0004917000865170008952F0008F52F0008AB
:1072000059300008B1300008093100084D3100083C
:1072100045320008211D000881180008551F00088C
:10722000E51D0008113B0008FD4D0008A1180008ED
:10723000AD180008B9180008D11B0008A13E0008CD
:10724000193F0008B543000841440008F36C0008EA
:10725000436D0008636D0008736D0008292700085E
:107260008517000871270008936D0008B36D0008AA
:10727000CB6D00089D270008C9270008B917000832
:10728000011A0008D5170008E917000811180008AE
:10729000CD49000821280008276E00084F6E00081D
:1072A000C51800080519000825190008511900081B
:1072B000F5440008214500085145000881450008B3
:1072C0007D190008A1190008311A0008691A000880
:1072D000D1190008A11A0008F11A0008991B00082A
:1072E000A91B0008ED240008114A0008091C000829
:1072F000D14A0008E14B000845460008594C0008F7
:10730000954C000801000000F810002088120020B1
:08731000C0110020006CDC023A
:10731800206861680834094204D0002202700130F4
:067328000139FBD17047A2
:10732E0020686168A2680C34124205D00B78037095
:0A733E0001300131013AF9D1704726
:04000005080069E79F
:00000001FF
